:100000000C94B9240C94EF240C94EF240C94E82A5B
:100010000C94EF240C94EF240C94EF240C94EF2414
:100020000C94EF240C94EF240C94EF240C94EF2404
:100030000C94EF240C94EF240C947A4A0C94EF2443
:100040000C94EF240C94EF240C94EF240C94EF24E4
:100050000C94D53A0C94EF240C94EF240C94EF24D8
:100060000C94EF240C94283D0C94EF240C94EF2472
:100070000C945F3D0C94EF240C94EF240C94EF242B
:100080000C94EF240C94EF240C94EF240C94B32ADA
:100090000C94EF240C94EF240C94EF240C94EF2494
:1000A0000C94EF240C94EF240C94EF240C94EF2484
:1000B0000C94522B0C94EF240C94EF240C94EF240A
:1000C0000C94EF240C94EF240C94EF240C94EF2464
:1000D0000C94EF240C94EF240C94EF240C94EF2454
:1000E0000C94EF240C94EF240C94963D0C94EF2484
:1000F0000C94EF240C94EF240C94EF240C94EF2434
:100100000C94EF240C941D2B0C94EF240C947E2A59
:100110000C94EF240C94EF240C94EF240C94EF2413
:100120000C94EF240C94EF240C94EF240C94EF2403
:100130000C94EF240C94FC240C94EF240C94EF24E6
:100140000C94EF240C94EF240C94EF240C94382599
:100150000C94EF240C94EF240C94EF240C94EF24D3
:100160000C94BA3C0C94EF240C94EF240C94F13CC6
:100170000C94EF240C94EF240C94EF240C94EF24B3
:100180000C94EF240C94EF240C94EF240C94EF24A3
:100190000C94EF240C94EF240C94EF240C94EF2493
:1001A0000C94EF240C94EF240C94EF240C94EF2483
:1001B0000C94EF240C94EF240C94EF240C94EF2473
:1001C0000C94EF240C94EF240C94EF240C94EF2463
:1001D0000C94EF240C94EF240C94EF240C94EF2453
:1001E0000C94EF240C94EF240C94EF240C94EF2443
:1001F0000C94EF240C94EF240C94EF24DE4F9D4FCD
:10020000A84FB84FC14F3A4F484F5C4F634F754F9F
:10021000844F8B4F974F494E5D4E6F4E744E844EB8
:10022000964EA84EB54EBA4ECA4EE14EEB4E004F1A
:10023000144F2A4F234B094C1B4C2B4C2E4C3C4C3F
:100240004C4C624C704C864C9A4CB54CC04CD54CC6
:10025000E54C004D0E4D274D3E4D534D5B4D6E4DC3
:10026000834D9E4DAC4DC14DD14DE84DF24D094EE3
:10027000194E2B4E374EE74FD24F384BCA53BF5310
:10028000AF53A65396538853775370535E535053CE
:1002900049533D532853175308530353F352E15224
:1002A000CF52C352BE52AE529A5290527C526B52AF
:1002B00058524B52385229521C5219520B52FB5170
:1002C000E851DA51C751B6519E5194517F516F5147
:1002D00055514751375121510E510451F050DB50C7
:1002E000C350B5509F508F5079506E505750475063
:1002F0003450265014500550D353DF530763423611
:10030000B79BD8A71A39685618AEBAAB558C1D3CA6
:10031000B7CC5763BD6DEDFD753EF6177231BF006A
:100320000000803F08000000BE922449123EABAAA4
:10033000AA2ABECDCCCC4C3E00000080BEABAAAAFF
:10034000AA3E00000000BF000000803F0000000047
:1003500000084178D3BB4387D1133D190E3CC3BD80
:100360004282AD2B3E68EC8276BED98FE1A93E4C2D
:1003700080EFFFBE01C4FF7F3F00000000000C942F
:1003800038520C94CA530C949F500C949E4D0C946C
:10039000D14D0C94AC4D0C94A84E0C9494510C94EB
:1003A000864C0C942B4E0C947C520C94534D0C9414
:1003B000A13B0C94274D0C94C7510C9428530C94DA
:1003C0009A4C0C94B54C0C94B84F0C94C14D0C94B1
:1003D0009E510C94384B0C94194E0C9496530C94DB
:1003E000DB500C94BA4E0C9426500C941C520C9476
:1003F00005500C943D530C94B13B0C940A540C944E
:1004000049530C94D54C0C94E8510C9429520C94FB
:10041000624C0C94634F0C9417530C94844F0C94BF
:10042000DF530C9447510C944B520C9434500C9461
:100430007F510C94F3520C940E510C948F500C94E9
:1004400014500C94A84F0C94FB510C94AF530C9483
:10045000E1520C94004F0C949A520C94B6510C94A7
:10046000844E0C9421510C94494E0C94D3530C940B
:10047000DE4F0C94E14E0C943C4C0C9488530C943D
:10048000F0500C942E4C0C94974F0C94E54C0C941B
:1004900057500C94BE520C94C93B0C94BF530C940F
:1004A0009D4F0C94A6530C945C4F0C9450530C9499
:1004B00077530C946E500C94374E0C94094C0C945A
:1004C00037510C94C3520C944C4C0C94744E0C94B5
:1004D00008530C94E84D0C94B54E0C942B4C0C9492
:1004E0002A4F0C9447500C943A4F0C94F24D0C94B4
:1004F000704C0C94FB3D0C94E93B0C94C3500C9451
:10050000E74F0C946F510C94B5500C9403530C941A
:10051000CF520C94484F0C9490520C9455510C941B
:10052000D24F0C94EB4E0C946B520C94094E0C94DD
:1005300079500C94F1240C946F4E0C94144F0C943D
:10054000004D0C94834D0C94754F0C943E4D0C94BF
:10055000C04C0C940B520C948B4F0C9419520C946D
:100560001B4C0C94AE520C94C14F0C945D4E0C94E9
:10057000DA510C946E4D0C945B4D0C9404510C9418
:10058000234B0C945E530C94F73B0C940E4D0C943F
:10059000CA4E0C9470530C94E7530C9458520C941C
:1005A000964E000038083A083C083E0878087A0859
:1005B00038093A093C093E0978097A09380A3A0AA1
:1005C0003C0A3E0A000102030405060708090A0B5B
:1005D000000001020300010001020300010001020A
:1005E0000300000000000000000000400840080078
:1005F0000000000000000040094009000000000069
:1006000000000000000008000800080008000000CA
:1006100000000900090009000900000000000A00AC
:100620000A000A000A0000000000000000000000AC
:100630000001020304050600000708090A0B0C006C
:10064000000D0E0F10000001020408102040800170
:10065000020408010204081020408001020408106E
:100660002040800102040801020101010101010191
:10067000010202020203030303030303030404044D
:100680000404040404050505050606000000062010
:1006900006400660068006E007090013001E0029D8
:1006A0000033003E00490053005E00690073007E85
:1006B00000890093009E00A800B300BE00C800D3CC
:1006C00000DD00E700F200FC00070111011B01261C
:1006D0000130013A0144014E01580163016D017777
:1006E0000180018A0194019E01A801B201BB01C5EC
:1006F00001CE01D801E101EB01F401FE0107021076
:1007000002190222022B0234023D0246024F025815
:10071000026002690271027A0282028A0293029BDB
:1007200002A302AB02B302BB02C302CA02D202D9C5
:1007300002E102E802F002F702FE0205030C0313D5
:10074000031A03210327032E0334033B034103470A
:10075000034D03530359035F0365036A0370037575
:10076000037A03800385038A038F03940398039D10
:1007700003A203A603AA03AF03B303B703BB03BFDC
:1007800003C203C603C903CD03D003D303D603D9E1
:1007900003DC03DF03E203E403E703E903EB03ED18
:1007A00003EF03F103F303F403F603F703F903FA8A
:1007B00003FB03FC03FD03FE03FE03FF03FF03FF34
:1007C00003FF03FF03FF03FF03FF03FF03FF03FE1A
:1007D00003FE03FD03FC03FB03FA03F803F703F630
:1007E00003F403F203F103EF03ED03EA03E803E686
:1007F00003E303E103DE03DB03D903D603D203CF14
:1008000003CC03C803C503C103BE03BA03B603B2D6
:1008100003AE03A903A503A0039C03970392038ED1
:1008200003890384037E03790374036E03690363FE
:10083000035D03570352034C0345033F033903335E
:10084000032C0325031F03180311030A030303FCEE
:1008500002F502EE02E602DF02D802D002C802C1AF
:1008600002B902B102A902A1029902910288028092
:100870000278026F0267025E0255024D0244023B9B
:100880000232022902200217020E020402FB01F2C8
:1008900001E801DF01D601CC01C201B901AF01A518
:1008A000019C01920188017E0174016A0160015678
:1008B000014C01420137012D01230119010E0104F0
:1008C00001FA00EF00E500DA00D000C500BB00B07F
:1008D00000A6009B00910086007B00710066005B13
:1008E00000510046003B00310026001B00100006AE
:1008F00000FBFFF0FFE6FFDBFFD0FFC6FFBBFFB052
:10090000FFA6FF9BFF90FF86FF7BFF70FF66FF5BEC
:10091000FF51FF46FF3CFF31FF27FF1CFF12FF077F
:10092000FFFDFEF3FEE8FEDEFED4FEC9FEBFFEB50F
:10093000FEABFEA1FE97FE8DFE83FE79FE6FFE6587
:10094000FE5BFE52FE48FE3EFE35FE2BFE22FE18EA
:10095000FE0FFE06FEFCFDF3FDEAFDE1FDD8FDCF36
:10096000FDC6FDBDFDB4FDABFDA3FD9AFD92FD8965
:10097000FD81FD78FD70FD68FD60FD58FD50FD486E
:10098000FD40FD38FD31FD29FD22FD1AFD13FD0C52
:10099000FD04FDFDFCF6FCEFFCE9FCE2FCDBFCD514
:1009A000FCCEFCC8FCC1FCBBFCB5FCAFFCA9FCA3A5
:1009B000FC9DFC98FC92FC8DFC87FC82FC7DFC7805
:1009C000FC73FC6EFC69FC65FC60FC5BFC57FC5333
:1009D000FC4FFC4BFC47FC43FC3FFC3BFC38FC342D
:1009E000FC31FC2EFC2BFC28FC25FC22FC1FFC1DF2
:1009F000FC1AFC18FC16FC14FC12FC10FC0EFC0C7F
:100A0000FC0BFC09FC08FC06FC05FC04FC03FC03D5
:100A1000FC02FC01FC01FC00FC00FC00FC00FC00F2
:100A2000FC00FC01FC01FC02FC02FC03FC04FC05D4
:100A3000FC06FC07FC08FC0AFC0BFC0DFC0FFC117F
:100A4000FC13FC15FC17FC19FC1CFC1EFC21FC24EF
:100A5000FC27FC29FC2DFC30FC33FC36FC3AFC3D29
:100A6000FC41FC45FC49FC4DFC51FC55FC5AFC5E2C
:100A7000FC63FC67FC6CFC71FC76FC7BFC80FC85F9
:100A8000FC8AFC90FC95FC9BFCA1FCA7FCACFCB296
:100A9000FCB9FCBFFCC5FCCBFCD2FCD8FCDFFCE6FF
:100AA000FCEDFCF3FCFAFC01FD09FD10FD17FD1F38
:100AB000FD26FD2EFD35FD3DFD45FD4DFD54FD5C46
:100AC000FD65FD6DFD75FD7DFD86FD8EFD97FD9F30
:100AD000FDA8FDB1FDB9FDC2FDCBFDD4FDDDFDE6F8
:100AE000FDEFFDF8FD02FE0BFE14FE1EFE27FE319B
:100AF000FE3AFE44FE4EFE57FE61FE6BFE75FE7F23
:100B0000FE89FE93FE9DFEA7FEB1FEBBFEC5FECF95
:100B1000FEDAFEE4FEEEFEF9FE03FF0DFF18FF22F3
:100B2000FF2DFF37FF42FF4CFF57FF61FF6CFF7740
:100B3000FF81FF8CFF96FFA1FFACFFB6FFC1FFCC8A
:100B4000FFD7FFE1FFECFFF7FF0000090011001ADB
:100B50000022002B0033003C0044004C0054005C99
:100B60000065006D0075007D0085008C0094009C80
:100B700000A400AB00B300BB00C200CA00D100D982
:100B800000E000E800EF00F600FD0005010C011395
:100B9000011A01210128012F0136013D0144014ABA
:100BA00001510158015F0165016C01720179017FFA
:100BB0000186018C01930199019F01A601AC01B24C
:100BC00001B801BE01C401CA01D001D601DC01E2B5
:100BD00001E801EE01F401F901FF0105020A02102A
:100BE0000216021B02210226022C02310236023CAE
:100BF00002410246024C02510256025B026002654B
:100C0000026A026F02740279027E02830288028DF8
:100C100002920297029B02A002A502A902AE02B3B1
:100C200002B702BC02C002C502C902CE02D202D67D
:100C300002DB02DF02E302E702EC02F002F402F858
:100C400002FC020003040308030D0310031403183D
:100C5000031C032003240328032C032F033303372F
:100C6000033A033E034203450349034D0350035433
:100C70000357035B035E036103650368036B036F44
:100C8000037203750379037C037F03820385038862
:100C9000038C038F039203950398039B039E03A188
:100CA00003A403A703A903AC03AF03B203B503B8BE
:100CB00003BA03BD03C003C203C503C803CA03CDFF
:100CC00003D003D203D503D703DA03DC03DF03E148
:100CD00003E403E603E803EB03ED03EF03F203F49D
:100CE00003F603F803FB03FD030004FC03EE03E03B
:100CF00003D203C503B703A9039C038F03810374C5
:100D00000367035A034D0340033303260319030CFF
:100D1000030003F302E602DA02CE02C102B502A921
:100D2000029D029002840278026C0261025502491F
:100D3000023D02320226021B020F020402F901EDFB
:100D400001E201D701CC01C101B601AB01A00195BF
:100D5000018B01800175016B01600156014B01415E
:100D60000137012C01220118010E010401FA00F0E3
:100D700000E600DC00D300C900BF00B600AC00A351
:100D8000009900900086007D0074006B006100589F
:100D9000004F0046003D0034002C0023001A0011D3
:100DA0000009000000F7FFEFFFE6FFDEFFD6FFCDF2
:100DB000FFC5FFBDFFB5FFACFFA4FF9CFF94FF8CF8
:100DC000FF84FF7CFF75FF6DFF65FF5DFF56FF4EE3
:100DD000FF46FF3FFF37FF30FF29FF21FF1AFF13B8
:100DE000FF0BFF04FFFDFEF6FEEFFEE8FEE1FEDA7C
:100DF000FED3FECCFEC5FEBEFEB7FEB1FEAAFEA32C
:100E0000FE9DFE96FE90FE89FE83FE7CFE76FE70C1
:100E1000FE69FE63FE5DFE57FE51FE4AFE44FE3E45
:100E2000FE38FE32FE2CFE26FE21FE1BFE15FE0FB6
:100E3000FE09FE04FEFEFDF9FDF3FDEDFDE8FDE219
:100E4000FDDDFDD7FDD2FDCDFDC7FDC2FDBDFDB869
:100E5000FDB2FDADFDA8FDA3FD9EFD99FD94FD8FA6
:100E6000FD8AFD85FD80FD7BFD77FD72FD6DFD68D2
:100E7000FD64FD5FFD5AFD56FD51FD4DFD48FD44ED
:100E8000FD3FFD3BFD36FD32FD2EFD29FD25FD21FB
:100E9000FD1DFD18FD14FD10FD0CFD08FD04FD00F9
:100EA000FDFCFCF8FCF4FCF0FCECFCE8FCE4FCE0F1
:100EB000FCDDFCD9FCD5FCD1FCCEFCCAFCC6FCC3D5
:100EC000FCBFFCBCFCB8FCB4FCB1FCAEFCAAFCA7AB
:100ED000FCA3FCA0FC9DFC99FC96FC93FC8FFC8C75
:100EE000FC89FC86FC83FC7FFC7CFC79FC76FC7333
:100EF000FC70FC6DFC6AFC67FC64FC61FC5EFC5CE5
:100F0000FC59FC56FC53FC50FC4EFC4BFC48FC4589
:100F1000FC43FC40FC3DFC3BFC38FC36FC33FC3124
:100F2000FC2EFC2CFC29FC27FC24FC22FC1FFC1DB5
:100F3000FC1BFC18FC16FC14FC11FC0FFC0DFC0B3C
:100F4000FC08FC0FFC1EFC2BFC39FC47FC55FC622A
:100F5000FC6FFC7DFC8AFC97FCA5FCB2FCBFFCCCC2
:100F6000FCD9FCE6FCF2FCFFFC0CFD18FD25FD3174
:100F7000FD3EFD4AFD56FD63FD6FFD7BFD87FD9344
:100F8000FD9FFDABFDB7FDC2FDCEFDDAFDE5FDF138
:100F9000FDFCFD07FE13FE1EFE29FE34FE3FFE4A49
:100FA000FE55FE60FE6BFE76FE81FE8BFE96FEA178
:100FB000FEABFEB6FEC0FECAFED5FEDFFEE9FEF3C6
:100FC000FEFDFE07FF11FF1BFF25FF2FFF38FF422D
:100FD000FF4CFF55FF5FFF69FF72FF7BFF85FF8EB0
:100FE000FF97FFA0FFAAFFB3FFBCFFC5FFCEFFD74F
:100FF000FFDFFFE8FFF1FFFAFF000000046F03CC02
:10100000038203B2038A039E038D038F038A038541
:101010000384037E037C037603760373036F036B01
:10102000036803640360035D035903560352034ED0
:10103000034B034703440340033C033903350332A6
:10104000032E032A032703230320031C031803157D
:101050000311030E030A0307030303FF02FC02F854
:1010600002F502F102EE02EA02E702E302E002DC2C
:1010700002D902D502D202CE02CB02C702C402C0FC
:1010800002BD02B902B602B202AF02AB02A802A4CC
:1010900002A1029D029A02960293028F028C02889C
:1010A00002850282027E027B027702740270026D68
:1010B000026902660263025F025C02580255025234
:1010C000024E024B024702440241023D023A0236FE
:1010D00002330230022C022902250222021F021BC7
:1010E000021802150211020E020B0207020402018D
:1010F00002FD01FA01F701F301F001ED01E901E65A
:1011000001E301DF01DC01D901D501D201CF01CC1E
:1011100001C801C501C201BE01BB01B801B501B1E1
:1011200001AE01AB01A701A401A1019E019A0197A3
:1011300001940191018D018A018701840180017D63
:10114000017A017701740170016D016A0167016321
:101150000160015D015A015701530150014D014ADF
:10116000014701440140013D013A01370134013199
:10117000012D012A012701240121011E011A011755
:1011800001140111010E010B01080104010101FE0E
:1011900000FB00F800F500F200EF00EC00E800E5CD
:1011A00000E200DF00DC00D900D600D300D000CD83
:1011B00000C900C600C300C000BD00BA00B700B43B
:1011C00000B100AE00AB00A800A500A2009F009CEB
:1011D000009900960092008F008C008900860083A1
:1011E0000080007D007A007700740071006E006B53
:1011F000006800650062005F005C00590056005303
:101200000050004D004A004700440041003F003CB0
:101210000039003600330030002D002A002700245A
:101220000021001E001B001800150012000F000C0A
:10123000000A00070004000100FEFFFBFFF8FFF5B5
:10124000FFF2FFEFFFEDFFEAFFE7FFE4FFE1FFDE64
:10125000FFDBFFD8FFD5FFD3FFD0FFCDFFCAFFC70D
:10126000FFC4FFC1FFBFFFBCFFB9FFB6FFB3FFB0B4
:10127000FFADFFABFFA8FFA5FFA2FF9FFF9CFF9A5A
:10128000FF97FF94FF91FF8EFF8CFF89FF86FF83FE
:10129000FF80FF7DFF7BFF78FF75FF72FF6FFF6DA3
:1012A000FF6AFF67FF64FF62FF5FFF5CFF59FF5645
:1012B000FF54FF51FF4EFF4BFF49FF46FF43FF40E6
:1012C000FF3EFF3BFF38FF35FF33FF30FF2DFF2A86
:1012D000FF28FF25FF22FF20FF1DFF1AFF17FF1524
:1012E000FF12FF0FFF0DFF0AFF07FF04FF02FFFFC2
:1012F000FEFCFEFAFEF7FEF4FEF2FEEFFEECFEEA66
:10130000FEE7FEE4FEE2FEDFFEDCFED9FED7FED401
:10131000FED2FECFFECCFECAFEC7FEC4FEC2FEBF9A
:10132000FEBCFEBAFEB7FEB4FEB2FEAFFEADFEAA34
:10133000FEA7FEA5FEA2FE9FFE9DFE9AFE98FE95CC
:10134000FE92FE90FE8DFE8BFE88FE85FE83FE8063
:10135000FE7EFE7BFE78FE76FE73FE71FE6EFE6CF8
:10136000FE69FE66FE64FE61FE5FFE5CFE5AFE578D
:10137000FE54FE52FE4FFE4DFE4AFE48FE45FE4321
:10138000FE40FE3EFE3BFE38FE36FE33FE31FE2EB4
:10139000FE2CFE29FE27FE24FE22FE1FFE1DFE1A45
:1013A000FE18FE15FE13FE10FE0EFE0BFE09FE06D5
:1013B000FE04FE01FEFFFDFCFDFAFDF7FDF5FDF26A
:1013C000FDF0FDEEFDEBFDE9FDE6FDE4FDE1FDDFF9
:1013D000FDDCFDDAFDD7FDD5FDD2FDD0FDCEFDCB88
:1013E000FDC9FDC6FDC4FDC1FDBFFDBDFDBAFDB813
:1013F000FDB5FDB3FDB0FDAEFDACFDA9FDA7FDA49F
:10140000FDA2FDA0FD9DFD9BFD98FD96FD94FD9127
:10141000FD8FFD8CFD8AFD88FD85FD83FD81FD7EB0
:10142000FD7CFD79FD77FD75FD72FD70FD6EFD6B38
:10143000FD69FD66FD64FD62FD5FFD5DFD5BFD58C0
:10144000FD56FD54FD51FD4FFD4DFD4AFD48FD4645
:10145000FD43FD41FD3FFD3CFD3AFD38FD35FD33CB
:10146000FD31FD2FFD2CFD2AFD28FD25FD23FD214D
:10147000FD1EFD1CFD1AFD18FD15FD13FD11FD0ED1
:10148000FD0CFD0AFD08FD05FD04FD00FDFFFCFB54
:10149000FCFBFCF7FCF4FCF8FCE8FCFDFCD6FC09CA
:1014A000FDBEFC1FFD89FC01FE0000FF03FF03FFE2
:1014B00003FF03FF03FF03FF03FF03FF03FF03FF1C
:1014C00003FF03FF03FF03FF03FF03FF03FF03FF0C
:1014D00003FF03FF03FF03FF03FF03FF03FF03FFFC
:1014E00003FF03FF03FF03FF03FF03FF03FF03FFEC
:1017000003000000FC00FC00FC00FC00FC00FC00EE
:10171000FC00FC00FC00FC00FC00FC00FC00FC00E9
:10172000FC00FC00FC00FC00FC00FC00FC00FC00D9
:10173000FC00FC00FC00FC00FC00FC00FC00FC00C9
:10174000FC00FC00FC00FC00FC00FC00FC00FC00B9
:10195000FC00FC00FC00FC00FC03001B00360053F4
:101960000071008F00AC00C700DF00F100FF00082D
:10197000010A0109010401FE00F900F500F400F775
:1019800000FD00060111011F012C013A014801551B
:101990000162016E01780181018601880185018063
:1019A0000176016901590147013501220110010247
:1019B00001F900F500FA000901220146017501ABA9
:1019C00001EA012C027102B502F70234036B039A9B
:1019D00003BF03D903E803EA03E103CE03B1038C99
:1019E00003610332030003CD029A0268023A020F38
:1019F00002E801C401A301850169014D012F011015
:101A000001ED00C7009E00740049002100FEFFE1C7
:101A1000FFCFFFC8FFCEFFE2FF03002F006400A14D
:101A200000E10024016501A401DD0111023D026213
:101A3000027F0293029F02A3029E0291027D026036
:101A4000023E021602E901B901870155012301F4A2
:101A500000C7009D0075004F0029000300DAFFB1A8
:101A6000FF85FF58FF2AFFFBFECBFE9AFE6BFE3C74
:101A7000FE0EFEE4FDBCFD98FD78FD5CFD45FD33EA
:101A8000FD25FD1EFD1BFD1EFD26FD31FD3FFD4E0E
:101A9000FD5EFD6DFD7BFD8AFD98FDA7FDB7FDC7D1
:101AA000FDD7FDE7FDF6FD06FE16FE27FE3BFE53C5
:101AB000FE71FE94FEBFFEF0FE26FF62FFA2FFE570
:101AC000FF29006C00AD00EA00220153017C019C5B
:101AD00001B201C001C401C001B501A50192017E9E
:101AE000016A01580148013C0133012D012A012AF4
:101AF000012E0135013F014B015901680175018338
:101B0000019101A001B101C601DF01FE0122024ADB
:101B10000275029F02C702EA0207031C0327032B78
:101B200003260319030503EA02C802A10275024550
:101B3000021202DE01AD017E01540130011101F9F2
:101B400000E600D600CC00C400C100C400CA00D624
:101B500000E600F9000F0125013A014D015E016C1C
:101B60000177018001850188018601810177016982
:101B700001570142012A011201FA00E200CA00B431
:101B8000009D00880072005D004900340021000FB4
:101B900000FFFFF1FFE4FFD7FFCBFFBFFFB4FFAAB9
:101BA000FFA2FF9DFF9CFF9EFFA4FFAEFFB8FFC3F7
:101BB000FFCCFFD2FFD6FFD7FFD5FFD3FFD0FFCB9F
:101BC000FFC6FFBDFFB0FF9DFF84FF63FF39FF0A23
:101BD000FFD5FE9DFE65FE2DFEFBFDCDFDA8FD8D16
:101BE000FD79FD70FD70FD78FD87FD99FDADFDC0AF
:101BF000FDD2FDE0FDEBFDF5FDFDFD05FE0EFE1841
:101C0000FE23FE2FFE3AFE43FE4AFE4EFE4FFE4DE1
:101C1000FE48FE40FE35FE26FE16FE05FEF4FDE7FC
:101C2000FDDEFDDDFDE5FDF6FD12FE39FE6AFEA2DC
:101C3000FEE1FE22FF62FF9FFFD7FF080032005542
:101C40000073008B009F00AF00BA00C200C500C443
:101C500000BF00B300A3008C006F004A002000F01A
:101C6000FFBBFF83FF4BFF15FFE5FEBBFE9AFE8423
:101C7000FE77FE74FE7BFE8AFEA0FEBBFEDBFE004E
:101C8000FF28FF53FF81FFB3FFE8FF2000590095B5
:101C900000D20010014E018A01C401FB012B025247
:101CA0000270028202880282027202580238021511
:101CB00002F101D001B2019A0188017B0174017225
:101CC000017401790181018A0194019E01A701B08B
:101CD00001BA01C501D201E401FA0113022F024C3D
:101CE0000267027F0292029E02A302A00296028570
:101CF000026F02530233021002EB01C4019C017314
:101D0000014A012001F400C8009B006D004100154C
:101D100000EBFFC4FFA1FF81FF67FF50FF3EFF31D3
:101D2000FF25FF1CFF13FF0AFF01FFF6FEE8FED6AA
:101D3000FEC1FEA7FE88FE66FE3FFE16FEEAFDBE61
:101D4000FD93FD6AFD44FD22FD03FDE8FCD1FCBBD3
:101D5000FCA6FC92FC7DFC68FC52FC3DFC29FC18B6
:101D6000FC0BFC03FC00FC05FC13FC2BFC4CFC787E
:101D7000FCAEFCEBFC30FD77FDBEFD05FE46FE82B1
:101D8000FEB6FEE2FE05FF1DFF2BFF2DFF25FF1215
:101D9000FFF7FED4FEA9FE7AFE47FE12FEDCFDA789
:101DA000FD75FD48FD21FD03FDECFCDEFCD7FCD6F6
:101DB000FCD9FCDFFCE7FCF0FCFAFC03FD0BFD1496
:101DC000FD1BFD23FD2BFD34FD3FFD4CFD5CFD7037
:101DD000FD86FD9FFDBCFDDBFDFCFD21FE47FE7089
:101DE000FE9AFEC5FEF0FE18FF3EFF5FFF79FF8DF5
:101DF000FF98FF9EFF9EFF9AFF94FF90FF90FF9435
:101E0000FFA0FFB1FFCBFFEAFF0600240043006004
:101E1000007D009B00BA00D900F80016013501557D
:101E20000176019601B501D401F301110230024E91
:101E3000026B028702A302BE02D802F1020903204C
:101E40000337034C036003730385039603A503B3B1
:101E500003BF03CB03D603E003E803EE03F403F868
:101E600003FC03FE0300040004FE03FB03F703F37B
:101E700003F103EE03E903E103D803D003C903C26E
:101E800003B903AE03A3039903900387037C036F95
:101E900003630358034E03430336032A031F03144B
:101EA000030A03FE02F202E602DC02D102C502B816
:101EB00002AC02A20298028D02810276026B0262DB
:101EC0000258024C02410237022D02240219020F6D
:101ED000020602FE01F401EA01E001D801D001C8C6
:101EE00001BE01B501AC01A5019D0195018D0185E2
:101EF000017E0177016F01680161015A0153014BB5
:101F00000145013E01380131012A0123011E01185A
:101F10000112010B010501FF00F900F300EE00E8DA
:101F200000E200DC00D500D000CB00C500C000B945
:101F300000B300AD00A700A2009C00960090008AAC
:101F40000084007F00790073006D00670061005C11
:101F50000056005000490043003D00380032002B7D
:101F60000025001F00190013000E0007000100FAF1
:101F7000FFF4FFEEFFE8FFE2FFDCFFD5FFCFFFC875
:101F8000FFC2FFBCFFB6FFB0FFA9FFA2FF9CFF97F7
:101F9000FF91FF8BFF84FF7EFF78FF71FF6BFF6572
:101FA000FF5FFF59FF53FF4DFF47FF41FF3BFF35E9
:101FB000FF2EFF28FF22FF1CFF16FF10FF09FF0363
:101FC000FFFDFEF8FEF2FEECFEE6FEDFFEDAFED4DA
:101FD000FECEFEC7FEC1FEBBFEB5FEAFFEA9FEA251
:101FE000FE9CFE96FE90FE8AFE84FE7EFE78FE71CA
:101FF000FE6AFE63FE5EFE58FE52FE4BFE44FE3E4F
:10200000FE38FE32FE2CFE25FE1EFE18FE12FE0CD1
:10201000FE05FEFFFDF9FDF2FDECFDE6FDDFFDD95D
:10202000FDD3FDCCFDC6FDC0FDBAFDB4FDADFDA6E2
:10203000FDA0FD9AFD95FD8FFD89FD82FD7CFD775C
:10204000FD72FD6CFD66FD60FD5BFD56FD52FD4DB4
:10205000FD47FD42FD3DFD39FD34FD30FD2CFD27E2
:10206000FD22FD1EFD1BFD18FD14FD10FD0CFD09DC
:10207000FD07FD05FD03FD01FDFEFCFCFCFBFCF97D
:10208000FCF8FCF7FCF7FCF7FCF6FCF7FCF7FCF8B7
:10209000FCF9FCFBFCFCFCFFFC01FD05FD08FD0C54
:1020A000FD11FD15FD1BFD21FD28FD2EFD36FD3E1C
:1020B000FD47FD52FD5DFD68FD73FD80FD8FFD9EBA
:1020C000FDAEFDBEFDCFFDE1FDF4FD08FE1CFE32C0
:1020D000FE49FE60FE78FE91FEAAFEC5FEE0FEFC13
:1020E000FE18FF35FF52FF71FF8FFFADFFCBFFEBF7
:1020F000FF0B002A00490067008500A300C100DF34
:1021000000FC00180134014F01690182019A01B1FC
:1021100001C701DC01F0010302150226023502436A
:102120000250025B0266026F0276027D0282028723
:10213000028A028D028E028E028D028A0288028538
:102140000280027A0274026D0266025E0255024B40
:1021500002410237022C02210215020902FD01F19F
:1021600001E401D801CB01BE01B001A201940187B5
:10217000017A016D015F0150014201360129011C04
:10218000010F010201F400E700DB00CE00C200B540
:1021900000A8009D00920087007C00700064005938
:1021A000004F0045003B00300026001C00130009D2
:1021B000000000F7FFEFFFE6FFDEFFD6FFCEFFC512
:1021C000FFBDFFB4FFACFFA5FF9EFF97FF8FFF870A
:1021D000FF80FF79FF74FF6DFF66FF5EFF58FF52BF
:1021E000FF4DFF46FF3FFF38FF32FF2DFF27FF2146
:1021F000FF1BFF14FF0FFF0AFF05FFFFFEF9FEF3B1
:10220000FEEEFEE8FEE2FEDCFED6FED1FECCFEC710
:10221000FEC1FEBBFEB6FEB1FEACFEA6FEA0FE9B5E
:10222000FE97FE92FE8CFE86FE81FE7CFE77FE739C
:10223000FE6EFE69FE63FE5FFE5AFE56FE52FE4EC5
:10224000FE49FE45FE41FE3DFE39FE35FE31FE2EC5
:10225000FE2BFE28FE25FE23FE20FE1EFE1CFE1A7F
:10226000FE19FE18FE17FE17FE17FE18FE19FE1ABD
:10227000FE1BFE1DFE1FFE22FE25FE29FE2EFE3445
:10228000FE3AFE40FE46FE4EFE56FE5FFE68FE72C1
:10229000FE7DFE89FE97FEA4FEB2FEC1FED1FEE2E7
:1022A000FEF4FE06FF18FF2DFF42FF58FF6EFF856C
:1022B000FF9DFFB6FFD0FFEBFF03000E00190023C8
:1022C000002E00380042004D00580062006D00777B
:1022D0000082008C009600A100AB00B500BF00C8D2
:1022E00000D200DC00E500EF00F80001010A011354
:1022F000011C0125012E0136013F01470150015803
:102300000160016801700178017F0187018E0196EB
:10231000019D01A401AC01B201B901C001C701CE08
:1023200001D401DB01E101E701ED01F301F901FF56
:102330000105020B02110216021C02210226022CC8
:1023400002310236023B02400245024A024F025469
:102350000259025E02620267026C02700275027923
:10236000027E02820287028B028F02940298029CF4
:1023700002A102A502A902AD02B202B602BA02BED1
:1023800002C202C602CA02CE02D202D602DA02DFBC
:1023900002E202E602EA02EE02F202F602FA02FEAD
:1023A000020103050309030C031003140317031BA5
:1023B000031E032203250328032B032F03320335B7
:1023C0000338033B033E0341034403460349034BE5
:1023D000034E0351035303560359035C035F036326
:1023E0000367036B036F03730378037D0383038821
:1023F000038E0394039A03A003A603AD03B303B9AA
:1024000003C003C603CC03D103D703DC03E103E518
:1024100003EA03EE03F103F403F703FA03FC03FDFD
:1024200003FE03FF03000400040004FF03FE03FD9A
:1024300003FC03FA03F803F603F303F103EE03EBE3
:1024400003E703E403E003DC03D803D403CF03CAA8
:1024500003C603C003BB03B603B003AA03A4039ED1
:1024600003980391038A0383037C0375036D03655B
:10247000035D0355034C0344033B03320328031F4E
:102480000315030B030103F702EC02E102D702CCB0
:1024900002C002B502AA029E02930287027B026F6B
:1024A00002630257024A023E023202250219020D5D
:1024B000020002F401E701DB01CE01C201B501A96E
:1024C000019D019001840178016C01600154014873
:1024D000013C013001240119010D010101F600EB5D
:1024E00000DF00D400C900BE00B300A8009D009327
:1024F0000088007E00730069005F0055004A0040BC
:102500000037002D002300190010000600FCFFF228
:10251000FFE9FFDFFFD5FFCBFFC1FFB7FFAEFFA491
:10252000FF9BFF91FF88FF7EFF75FF6CFF62FF59E5
:10253000FF50FF47FF3EFF35FF2CFF23FF1AFF111F
:10254000FF08FFFFFEF7FEEEFEE5FEDDFED4FECB4C
:10255000FEC3FEBAFEB1FEA9FEA0FE98FE8FFE8667
:10256000FE7EFE75FE6DFE64FE5CFE53FE4AFE427C
:10257000FE39FE31FE28FE1FFE17FE0EFE06FEFD92
:10258000FDF4FDECFDE3FDDBFDD2FDCAFDC1FDB8B0
:10259000FDB0FDA7FD9FFD96FD8EFD85FD7DFD74C3
:1025A000FD6CFD64FD5BFD53FD4BFD43FD3BFD33C9
:1025B000FD2BFD23FD1BFD13FD0BFD04FDFCFCF5B8
:1025C000FCEDFCE6FCDFFCD8FCD1FCCAFCC3FCBD86
:1025D000FCB6FCB0FCAAFCA3FC9DFC98FC92FC8C15
:1025E000FC87FC82FC7CFC78FC73FC6EFC6AFC655E
:1025F000FC61FC5DFC5AFC56FC53FC4FFC4CFC4956
:10260000FC47FC44FC42FC40FC3EFC3CFC3BFC39EF
:10261000FC38FC37FC37FC36FC36FC35FC35FC3628
:10262000FC36FC37FC37FC38FC39FC3BFC3CFC3E00
:10263000FC3FFC41FC44FC46FC48FC4BFC4EFC507F
:10264000FC54FC57FC5AFC5EFC61FC65FC69FC6DAB
:10265000FC71FC75FC79FC7EFC82FC87FC8CFC9098
:10266000FC95FC9AFC9FFCA4FCAAFCAFFCB4FCBA51
:10267000FCBFFCC4FCCAFCD0FCD5FCDBFCE0FCE6E7
:10268000FCECFCF2FCF7FCFDFC02FD08FD0DFD116D
:10269000FD16FD1AFD1EFD21FD24FD26FD28FD2A47
:1026A000FD2BFD2CFD2CFD2DFD2DFD2DFD2CFD2CE0
:1026B000FD2CFD2BFD2BFD2BFD2BFD2BFD2BFD2CD8
:1026C000FD2DFD2EFD30FD32FD34FD37FD3AFD3D83
:1026D000FD41FD45FD4AFD4EFD54FD59FD5FFD6583
:1026E000FD6BFD72FD78FD7FFD86FD8DFD95FD9CEA
:1026F000FDA4FDABFDB3FDBBFDC3FDCBFDD3FDDBF9
:10270000FDE3FDECFDF4FDFCFD05FE0EFE16FE1FD7
:10271000FE28FE31FE3AFE43FE4DFE56FE5FFE6988
:10272000FE73FE7DFE87FE91FE9BFEA6FEB0FEBB05
:10273000FEC5FED0FEDBFEE6FEF1FEFDFE08FF1349
:10274000FF1FFF2AFF36FF41FF4DFF58FF64FF7058
:10275000FF7BFF87FF92FF9EFFA9FFB5FFC0FFCC65
:10276000FFD7FFE2FFEDFFF8FF0000030010002994
:10277000003C004900550061006F0082009A00B3E0
:1027800000C600D500E200EA00EC00E700E400E348
:1027900000DF00D900D100CC00C500B900AC009F1B
:1027A000009300860079006D00650060006000679E
:1027B0000075008A00A700CA00F3001F014C0175D4
:1027C000019701B401D101EF010C02250238024446
:1027D000024A024D024D024B024A024E025A026D5B
:1027E0000285029E02B802D502FA02250353037D38
:1027F00003A503C903E703FB030004FA03EC03DBAF
:1028000003C603AF03990389037C036F0360034C82
:102810000336031D030203E702CF02BB02AB029D96
:102820000291028302730262024E02390222020BFB
:1028300002F501DE01C701B2019E018D017A01633B
:102840000148012C010D01ED00C900A4007F005BCF
:102850000036001000E8FFBFFF97FF6FFF4BFF2D12
:10286000FF15FFFFFEEEFEE4FEDFFED7FEC6FEB262
:10287000FE9BFE81FE5FFE36FE0EFEE6FDBDFD8F79
:10288000FD5EFD2DFDFFFCD6FCB6FC9BFC84FC73BD
:10289000FC6AFC69FC6EFC7AFC8BFC9FFCB1FCBD05
:1028A000FCC4FCC9FCCEFCD5FCDEFCE9FCF6FC0259
:1028B000FD07FD05FDFDFCF2FCE6FCD9FCCFFCC7E5
:1028C000FCC0FCBBFCBAFCBFFCCAFCDAFCF3FC1489
:1028D000FD3AFD5CFD79FD95FDB2FDCFFDEAFDFE03
:1028E000FD06FEFEFDEAFDD6FDC3FDB2FDA0FD8D99
:1028F000FD7CFD6EFD68FD68FD6BFD70FD7AFD8A57
:10290000FDA0FDB5FDC9FDDCFDEDFDFBFD06FE13E3
:10291000FE23FE33FE43FE52FE5FFE6BFE77FE8516
:10292000FE93FEA3FEB4FEC4FED3FEE6FEFDFE1340
:10293000FF26FF34FF45FF5EFF81FFA9FFD3FFFBAA
:10294000FF1F003B004E005B00660070007E008FA2
:1029500000A500BB00CC00D800E000E600EE00F9C6
:1029600000070111011501160113010B01FE00EF13
:1029700000E400DC00D500CD00C300B900AC009F2E
:102980000094008F008F008C00880080007400632A
:10299000004C0030001200F4FFD6FFBBFFA4FF8FF5
:1029A000FF7DFF6EFF63FF5AFF54FF51FF54FF5E30
:1029B000FF6AFF76FF81FF89FF89FF82FF76FF6E46
:1029C000FF6BFF69FF64FF5CFF59FF57FF54FF4F28
:1029D000FF4DFF52FF59FF62FF73FF8EFFADFFC92E
:1029E000FFE4FF01002100440067008800A200B05E
:1029F00000BE00CE00DF00E400D700C900C000C563
:102A000000C200B800AD00B200C700DD00E800E57C
:102A100000E700EF00FF00050102010101060115BA
:102A2000012F014A015B0158015401680178017BC3
:102A3000016C0164016D0174017D0187018A0188C7
:102A4000018B01910196019101A101CB01ED0105DD
:102A50000215023102480247023B0234023E02588C
:102A600002750280027A026C0270027F0284027B8D
:102A7000026702510242023A022B020E02E901DF12
:102A800001E101DA01BC018D016601460134013624
:102A9000013B0132011A01FE00E900C20089004831
:102AA000000F00E5FFC1FFA1FF80FF61FF4BFF4565
:102AB000FF45FF4BFF58FF75FF9DFFBFFFDFFFFF87
:102AC000FF1D0033003C0040004200430040003640
:102AD0000024000B00F4FFE9FFEAFFF1FFF7FFFD20
:102AE000FF0D002D0057008100A300BD00DE00098E
:102AF0000139015D01700179017501660146011915
:102B000001E200A50067002E00F9FFC4FF8FFF60FF
:102B1000FF3AFF17FFF8FEDFFECEFEC3FEBCFEB499
:102B2000FEA5FE8BFE6CFE4BFE27FEFEFDD1FDAA30
:102B3000FD87FD63FD3FFD1DFD01FDEBFCE0FCE1BC
:102B4000FCEAFCF8FC10FD30FD4FFD64FD75FD92C4
:102B5000FDB6FDDDFD01FE20FE3DFE55FE67FE7566
:102B6000FE7EFE86FE8FFE9BFEAAFEBBFECCFEDC3A
:102B7000FEE9FEF8FE0CFF24FF3BFF4EFF67FF88D7
:102B8000FFABFFC8FFDCFFECFFFAFF06000B0006FF
:102B900000F6FFE2FFD1FFC6FFBCFFB4FFB1FFB2FA
:102BA000FFB7FFBDFFC5FFD0FFE4FF0100280051C4
:102BB0000075009600AE00BC00BD00B400A90095F1
:102BC000007D00680058004E003F002F001F000EDF
:102BD00000FEFFEFFFE6FFE5FFE7FFEBFFF0FFF191
:102BE000FFEEFFEBFFE7FFE0FFD3FFC8FFC0FFB83A
:102BF000FFABFF9AFF8CFF84FF82FF83FF87FF8D6F
:102C0000FF94FF9DFFA7FFB3FFBFFFCBFFD6FFE100
:102C1000FFEBFFF4FFFBFFFDFF07000B000F0013AE
:102C200000150013000E00090008000A000C001037
:102C30000019002C0049006F009F00D7000C013FD5
:102C4000017401AF01EB012A026B02AA02E6022025
:102C50000354038503B203D503EE03FD030004FB15
:102C600003EB03D003AF038A03600333030103C8FC
:102C7000028F0256022002EA01BA018E0163013C72
:102C8000011A01FC00E500D700D100D400DD00EE00
:102C90000007012501480171019D01C801F3011AD6
:102CA00002400264028902AC02CF02EC02FF020A77
:102CB000031103150316031603160316031703184F
:102CC00003190319031C0322032B033203360337B2
:102CD0000335032F03250316030203EA02CD02AADC
:102CE0000285025D0230020402D601A30170013B9D
:102CF000010501CC00970064003100FCFFC3FF8791
:102D0000FF4DFF15FFDAFEA1FE6BFE3BFE13FEF347
:102D1000FDD9FDC4FDB5FDA9FDA0FD9AFD95FD936E
:102D2000FD95FD9AFD9FFDA6FDACFDB1FDB6FDBA7A
:102D3000FDBDFDC0FDC4FDCBFDD1FDD5FDD6FDD64D
:102D4000FDD4FDD1FDCBFDC2FDB7FDADFDA1FD93D1
:102D5000FD83FD70FD5CFD48FD33FD1DFD08FDF4A8
:102D6000FCE1FCD1FCC5FCBCFCB6FCB3FCB3FCB57F
:102D7000FCBBFCC3FCD1FCE3FCF8FC11FD2CFD4CBE
:102D8000FD72FD9AFDC4FDEEFD19FE42FE6BFE9440
:102D9000FEBBFEE1FE07FF2BFF4DFF6EFF8CFFA683
:102DA000FFBBFFCCFFD8FFDFFFE2FFE3FFE2FFDF67
:102DB000FFDBFFD6FFCFFFC7FFBFFFB6FFACFFA112
:102DC000FF96FF89FF7CFF6EFF5FFF4DFF3AFF28F4
:102DD000FF18FF08FFF9FEEAFEDCFECEFEC1FEB6DC
:102DE000FEAEFEABFEAFFEBAFECAFEDCFEF4FE1384
:102DF000FF39FF5FFF84FFABFFD3FFFEFF2B0056C1
:102E0000008000AB00D200F7001A013C015A0174A7
:102E1000018B019D01AC01B801C101C601CA01CC01
:102E200001CD01CC01CA01C701C301BD01B601AE8C
:102E300001A4019C0194018B017F01720163015285
:102E40000141013201230114010401F400E600DC18
:102E500000D400CD00C500BF00BC00BB00BC00BD5D
:102E600000BE00BF00BF00BE00BC00B800B400B28E
:102E700000B000AB00A3009C00960091008D00887C
:102E800000840080007C007900780077007700776C
:102E90000079007D0083008A0094009F00AB00B998
:102EA00000C700D500E300F100FF000D0119012467
:102EB000012B0131013201300128011D010E01FDFC
:102EC00000E800CF00B40097007A005E0043002BBA
:102ED000001400FEFFE8FFD7FFCBFFC3FFC2FFC80F
:102EE000FFD1FFDDFFEBFFFEFF13002A004000557E
:102EF000006B0081009700AB00BC00CB00D600DF68
:102F000000E400E400E200DF00DA00D500CF00C8F2
:102F100000C000B900B200AC00A600A300A300A44A
:102F200000A500A300A1009F009E009B00970092B7
:102F3000008A00810077006B005F0050003F002D89
:102F4000001C000B00FBFFEBFFDCFFCFFFC4FFBB4F
:102F5000FFB6FFB5FFB7FFBBFFC1FFC9FFD3FFDD62
:102F6000FFE6FFF0FFFAFF03000C0012001500154A
:102F700000130010000B000500FEFFF5FFEAFFE064
:102F8000FFD5FFCBFFC0FFB5FFAAFF9FFF96FF8EC7
:102F9000FF88FF83FF7FFF7CFF7BFF7DFF81FF8634
:102FA000FF8BFF8FFF94FF98FF9EFFA5FFAEFFB73B
:102FB000FFBEFFC4FFC9FFCDFFD1FFD6FFDAFFDEA2
:102FC000FFE1FFE3FFE6FFE9FFEDFFF2FFF6FFFAA7
:102FD000FFFCFFFCFFFBFFF8FFF7FFF8FFFAFFFB2A
:102FE000FFFAFFF8FFF6FFF4FFF2FFEFFFEBFFE55C
:102FF000FFDDFFD3FFCAFFC0FFB6FFADFFA2FF9307
:10300000FF80FF6EFF5DFF4FFF43FF3AFF34FF314C
:10301000FF32FF34FF35FF37FF39FF3CFF40FF44ED
:10302000FF48FF4BFF4CFF4AFF48FF45FF41FF3D74
:10303000FF38FF30FF25FF17FF06FFF1FEDAFEC164
:10304000FEA5FE88FE69FE48FE27FE06FEE6FDCAD6
:10305000FDB2FD9BFD84FD70FD5EFD4EFD44FD4116
:10306000FD44FD4EFD5EFD73FD8CFDA8FDC8FDED2C
:10307000FD13FE37FE59FE78FE9AFEBFFEDEFEF619
:10308000FE08FF15FF1DFF1FFF1FFF1AFF0FFFFEAA
:10309000FEE8FECFFEB5FE9CFE87FE75FE65FE5681
:1030A000FE4AFE44FE44FE4CFE5EFE78FE93FEB0F9
:1030B000FECEFEEFFE13FF37FF57FF74FF8FFFA812
:1030C000FFBFFFD7FFECFFFDFF0C001F00310043E7
:1030D000005600680079008B009D00AE00BF00D054
:1030E00000E100F100020112012101310140014F14
:1030F000015E016D017B0189019701A401B101BE4F
:1031000001CB01D701E301EF01FB01060211021C13
:1031100002260231023B0245024E02580261026A57
:103120000273027C0284028D0295029D02A502AC0C
:1031300002B402BB02C202CA02D102D802DF02E517
:1031400002EC02F302F902000307030D0313031A52
:1031500003200326032C03320338033E0344034AAF
:1031600003500356035C03610367036D0372037826
:10317000037D03820387038C03910396039A039FC5
:1031800003A303A703AB03AF03B303B703BB03BEA0
:1031900003C203C503C803CB03CE03D103D403D6B4
:1031A00003D903DB03DE03E003E203E403E603E801
:1031B00003E903EB03EC03EE03EF03F003F103F287
:1031C00003F303F403F403F503F503F503F503F543
:1031D00003F503F403F403F303F203F103F003EF45
:1031E00003EE03EC03EB03E903E803E603E403E285
:1031F00003E003DE03DC03D903D703D403D203CFF8
:1032000003CC03C803C503C103BD03B903B503B1B0
:1032100003AC03A703A2039D03970392038C0386C9
:103220000380037A0373036C0366035E0357035042
:103230000348034003390330032803200317030E18
:10324000030503FC02F302EA02E002D602CC02C349
:1032500002B802AE02A4029A028F0285027B0270BB
:103260000265025B02500246023B02300225021B4D
:103270000210020402F901EE01E201D601CA01BD09
:1032800001B101A50198018C017F0173016601590B
:10329000014D01410135012A011E0113010801FD03
:1032A00000F300E900DF00D500CB00C100B700AD9E
:1032B00000A4009A00900086007C00730069006002
:1032C0000056004D0044003B003200290020001849
:1032D00000100008000000F8FFF1FFE9FFE2FFDB4B
:1032E000FFD4FFCEFFC7FFC1FFBAFFB4FFAEFFA8F8
:1032F000FFA2FF9CFF96FF91FF8BFF86FF80FF7B65
:10330000FF76FF71FF6DFF68FF64FF60FF5CFF5891
:10331000FF55FF52FF4EFF4BFF48FF44FF41FF3E6A
:10332000FF3AFF36FF33FF2FFF2AFF26FF21FF1C46
:10333000FF18FF13FF0EFF09FF04FFFFFEFAFEF563
:10334000FEF1FEECFEE8FEE3FEDFFEDBFED7FED381
:10335000FED0FECCFEC8FEC4FEC1FEBDFEB9FEB569
:10336000FEB2FEAEFEAAFEA6FEA2FE9FFE9BFE974A
:10337000FE94FE90FE8DFE89FE86FE83FE80FE7D1D
:10338000FE7AFE77FE74FE72FE6FFE6DFE6AFE68C8
:10339000FE66FE64FE62FE60FE5EFE5DFE5BFE5A41
:1033A000FE58FE57FE56FE54FE54FE53FE52FE518A
:1033B000FE51FE50FE50FE50FE50FE50FE51FE519A
:1033C000FE51FE52FE53FE53FE54FE55FE56FE576E
:1033D000FE58FE59FE5AFE5BFE5CFE5EFE5FFE601E
:1033E000FE61FE63FE64FE65FE66FE68FE69FE6ABF
:1033F000FE6BFE6CFE6DFE6EFE6FFE6FFE70FE716C
:10340000FE71FE72FE73FE73FE73FE74FE74FE7434
:10341000FE74FE74FE74FE74FE74FE73FE73FE7220
:10342000FE71FE6FFE6EFE6CFE69FE67FE64FE615D
:10343000FE5EFE5AFE56FE52FE4EFE4AFE45FE401F
:10344000FE3BFE36FE31FE2CFE26FE21FE1BFE1547
:10345000FE0FFE08FE02FEFBFDF4FDEDFDE7FDE0C4
:10346000FDD8FDD1FDCAFDC2FDBAFDB3FDABFDA384
:10347000FD9BFD92FD89FD81FD78FD6EFD65FD5B87
:10348000FD51FD46FD3CFD32FD27FD1CFD11FD06F5
:10349000FDFBFCF0FCE5FCDBFCD0FCC5FCBBFCB19F
:1034A000FCA7FC9DFC93FC8AFC80FC77FC6EFC6511
:1034B000FC5DFC55FC4EFC46FC3FFC39FC33FC2D0E
:1034C000FC28FC22FC1EFC19FC15FC11FC0EFC0A5D
:1034D000FC07FC04FC02FC00FC00FC00FC00FC00FF
:1034E000FC00FC00FC00FC00FC00FC00FC00FC00FC
:1034F000FC03FC07FC0BFC10FC15FC1BFC22FC294C
:10350000FC30FC38FC41FC49FC53FC5CFC67FC7162
:10351000FC7CFC88FC93FCA0FCADFCBAFCC7FCD591
:10352000FCE3FCF2FC01FD10FD20FD30FD40FD51EF
:10353000FD62FD73FD84FD96FDA8FDBAFDCCFDDFA7
:10354000FDF2FD05FE18FE2BFE3EFE52FE65FE78E6
:10355000FE8BFE9FFEB3FEC6FEDAFEEEFE01FF15F9
:10356000FF29FF3CFF50FF63FF76FF89FF9CFFAF01
:10357000FFC2FFD5FFE8FFFAFF0700100019002384
:10358000002E00390043004D0056005F0067006EBA
:1035900000740079007D008100850089008D009213
:1035A0000097009D00A300A800AD00B100B500B7D2
:1035B00000B800B900B900B900B900B800B800B847
:1035C00000BA00BB00BD00C000C300C500C800CAEF
:1035D00000CC00CE00D000D200D400D700DB00DF4A
:1035E00000E400E900EF00F600FE0005010D011403
:1035F000011B01210127012C01320137013C01424D
:103600000147014D01520158015D01610166016AE6
:10361000016D016F0171017301740175017601770C
:1036200001780179017C017E018101850188018C8D
:10363000018F0191019301940195019601960197E3
:103640000198019A019C019F01A201A601AA01AF64
:1036500001B301B801BD01C201C801CD01D301D838
:1036600001DD01E201E701EC01F101F601FB0101DD
:103670000207020D0214021C0224022C0234023D35
:103680000246024F0258026002690271027A028306
:10369000028C0294029D02A402AC02B302BA02C1DF
:1036A00002C702CE02D602DD02E502ED02F402FB01
:1036B00002010308030D03130319031F0325032D40
:1036C0000334033D0346034E0357035F036803704F
:1036D000037803800387038D0394039A03A003A751
:1036E00003AD03B303BA03C103C803CF03D603DD9D
:1036F00003E303E803ED03F103F403F603F803FA2D
:1037000003FB03FD03FE03FF0300040004FF03FDAE
:1037100003FA03F603F203EE03E903E403DE03D83E
:1037200003D103CA03C203BA03B203AB03A4039ECB
:1037300003990394038F038C038803850382037E1C
:10374000037B037803750371036D036803640360EF
:10375000035C035903550352034F034C03480343CF
:10376000033E03380331032A03210319030F030522
:1037700003FB02F002E402D802CC02BE02AF02A0B8
:10378000028F027E026C025902460232021F020BB5
:1037900002F701E401D001BD01AA0198018601757B
:1037A00001640153014201320120010F01FE00EDCD
:1037B00000DB00C900B700A400920080006D005B30
:1037C0000049003600250014000400F3FFE4FFD692
:1037D000FFC8FFBBFFAEFFA2FF97FF8DFF84FF7BFB
:1037E000FF73FF6CFF65FF60FF5AFF55FF51FF4DF0
:1037F000FF49FF47FF44FF43FF43FF42FF43FF43AF
:10380000FF44FF44FF43FF41FF3EFF3BFF37FF33D1
:10381000FF2FFF2CFF29FF26FF23FF21FF1EFF1A8A
:10382000FF17FF12FF0DFF08FF02FFFCFEF5FEEF82
:10383000FEE8FEE0FED8FED1FEC8FEC0FEB7FEAF39
:10384000FEA6FE9DFE94FE8CFE84FE7DFE76FE703E
:10385000FE6BFE66FE62FE5FFE5CFE5AFE58FE5781
:10386000FE56FE56FE55FE54FE52FE50FE4EFE4CD7
:10387000FE49FE47FE44FE41FE3FFE3CFE39FE3659
:10388000FE32FE2EFE2AFE26FE23FE1FFE1CFE1921
:10389000FE16FE12FE0EFE0AFE06FE01FEFDFDF8FD
:1038A000FDF3FDEFFDEBFDE7FDE3FDDFFDDCFDD905
:1038B000FDD5FDD2FDCEFDCAFDC7FDC2FDBEFDBBDF
:1038C000FDB7FDB4FDB1FDAEFDAAFDA6FDA2FD9CB8
:1038D000FD96FD8FFD88FD82FD7CFD76FD71FD6D01
:1038E000FD68FD61FD5BFD53FD4AFD40FD36FD2B8E
:1038F000FD22FD19FD10FD08FD01FDFAFCF3FCECB5
:10390000FCE4FCDCFCD3FCCAFCC0FCB6FCACFCA1B7
:10391000FC98FC8FFC87FC7FFC79FC73FC6EFC69D7
:10392000FC65FC62FC5FFC5DFC5CFC5BFC5AFC5AC9
:10393000FC5AFC5BFC5BFC5CFC5CFC5CFC5CFC5CCB
:10394000FC5BFC59FC57FC55FC52FC4FFC4CFC4901
:10395000FC46FC42FC3FFC3BFC37FC34FC30FC2CBE
:10396000FC28FC25FC22FC20FC1EFC1DFC1CFC1C75
:10397000FC1CFC1CFC1CFC1DFC1FFC20FC22FC2570
:10398000FC28FC2CFC31FC36FC3CFC43FC4BFC547E
:10399000FC5EFC68FC72FC7DFC88FC93FC9EFCAA2F
:1039A000FCB5FCC0FCCBFCD5FCE0FCEAFCF4FCFE66
:1039B000FC08FD11FD1BFD24FD2EFD37FD40FD49DA
:1039C000FD51FD5AFD62FD69FD70FD77FD7DFD83B2
:1039D000FD8AFD90FD98FD9FFDA8FDB1FDBAFDC4D7
:1039E000FDCEFDD9FDE4FDF0FDFCFD09FE17FE2630
:1039F000FE34FE44FE53FE63FE73FE83FE94FEA57A
:103A0000FEB7FEC8FEDAFEEDFE00FF12FF26FF380D
:103A1000FF4BFF5DFF70FF83FF94FFA6FFB7FFC75B
:103A2000FFD7FFE6FFF3FFFEFF030017002B004068
:103A300000540068007D009100A500B900CD00E1B0
:103A400000F50008011B012E0141015301650177BA
:103A50000189019B01AC01BE01CF01E001F101022E
:103A600002130223023402440254026502750284E6
:103A7000029402A302B202C102CF02DD02EA02F8FE
:103A800002040311031D03280333033E03480352BA
:103A9000035C0365036F0377038003890391039934
:103AA00003A103A903B103B903C003C803CF03D51E
:103AB00003DC03E103E703EC03F003F403F803FA88
:103AC00003FD03FE03FF03000400040004FF03FEE4
:103AD00003FC03FA03F803F603F403F103EF03EC2A
:103AE00003EA03E703E403E203DF03DC03D903D5BE
:103AF00003D203CE03C903C503C003BA03B403AEA4
:103B000003A703A0039803900388037F0376036D44
:103B10000363035A03500345033B03310326031B8E
:103B20000311030603FB02F002E502D902CE02C232
:103B300002B602AA029D0291028402760269025B29
:103B4000024E0240023202240216020802FA01EC7E
:103B500001DE01D001C201B501A7019A018D0180EA
:103B6000017301660159014C01400133012601191D
:103B7000010B01FE00F000E200D400C500B600A772
:103B800000980089007A006B005B004C003D002E1D
:103B9000001F0011000200F4FFE6FFD9FFCBFFBFBA
:103BA000FFB2FFA6FF9AFF8FFF84FF7AFF70FF66C8
:103BB000FF5CFF54FF4BFF43FF3BFF33FF2CFF2510
:103BC000FF1EFF18FF11FF0BFF06FF01FFFCFEF7B2
:103BD000FEF2FEEEFEEAFEE6FEE2FEDFFEDCFED9CF
:103BE000FED6FED4FED1FECFFECDFECBFECAFEC871
:103BF000FEC7FEC6FEC5FEC5FEC4FEC4FEC4FEC5AD
:103C0000FEC5FEC6FEC8FEC9FECCFECEFED1FED469
:103C1000FED8FEDCFEE0FEE4FEE9FEEFFEF4FEFA76
:103C2000FEFFFE05FF0BFF11FF17FF1DFF23FF29FE
:103C3000FF2EFF33FF37FF3BFF3FFF42FF44FF46AE
:103C4000FF47FF47FF47FF46FF45FF42FF3FFF3B60
:103C5000FF37FF32FF2CFF25FF1EFF17FF0FFF0668
:103C6000FFFDFEF3FEE9FEDFFED4FEC9FEBEFEB29E
:103C7000FEA7FE9BFE8EFE82FE75FE68FE5BFE4E7C
:103C8000FE40FE32FE24FE16FE07FEF9FDEAFDDBD5
:103C9000FDCCFDBDFDADFD9EFD8EFD7FFD6FFD608C
:103CA000FD50FD41FD31FD22FD13FD04FDF6FCE854
:103CB000FCDAFCCDFCC0FCB4FCA8FC9DFC93FC8AA7
:103CC000FC81FC79FC73FC6DFC68FC64FC61FC5FAE
:103CD000FC5EFC5FFC60FC63FC68FC6DFC74FC7CBF
:103CE000FC85FC8FFC9BFCA8FCB6FCC5FCD6FCE864
:103CF000FCFBFC0FFD24FD3AFD51FD69FD82FD9C9E
:103D0000FDB6FDD2FDEEFD0BFE28FE46FE64FE83F1
:103D1000FEA3FEC2FEE2FE03FF23FF44FF64FF8515
:103D2000FFA6FFC7FFE7FF080028004800680088DB
:103D300000A700C600E40002011F013B0157017209
:103D4000018D01A601BF01D701EF0105021A022F63
:103D500002430255026702780288029602A402B169
:103D600002BD02C802D202DA02E202E902EF02F365
:103D700002F702FA02FB02FC02FB02FA02F702F46B
:103D800002F002EA02E402DD02D502CC02C202B76E
:103D900002AC029F02920285027602670257024736
:103DA00002350223021102FE01EA01D601C201AC72
:103DB00001970181016B0154013D0126010F01F7BB
:103DC00000DF00C700AF0096007E0065004C0033A6
:103DD000001A000200E9FFD0FFB7FF9FFF86FF6EC9
:103DE000FF56FF3EFF26FF0EFFF7FEE0FEC9FEB3C3
:103DF000FE9DFE87FE71FE5CFE47FE33FE1EFE0B3F
:103E0000FEF7FDE4FDD1FDBFFDADFD9BFD8AFD7913
:103E1000FD69FD59FD4AFD3BFD2DFD1FFD11FD0412
:103E2000FDF8FCECFCE1FCD6FCCCFCC2FCB9FCB11E
:103E3000FCA9FCA2FC9BFC94FC8FFC89FC85FC810A
:103E4000FC7DFC7AFC77FC75FC73FC72FC72FC72E6
:103E5000FC72FC73FC74FC77FC79FC7CFC80FC84B9
:103E6000FC89FC8EFC94FC9AFCA1FCA8FCAFFCB77E
:103E7000FCC0FCC8FCD1FCDBFCE5FCEFFCF9FC045D
:103E8000FD10FD1BFD27FD33FD40FD4DFD5BFD6875
:103E9000FD77FD85FD94FDA4FDB4FDC4FDD4FDE5D5
:103EA000FDF6FD07FE19FE2AFE3CFE4EFE60FE7387
:103EB000FE85FE97FEAAFEBCFECFFEE2FEF5FE08E2
:103EC000FF1BFF2EFF41FF55FF68FF7CFF90FFA502
:103ED000FFB9FFCDFFE1FFF2FF0200060009000D70
:103EE000001000140017001A001E002100250028F1
:103EF000002C002F003300360039003D0040004305
:103F00000047004A004E005100550058005C005F19
:103F1000006200660069006D007000730077007A2F
:103F2000007E008100850088008B008F0092009643
:103F30000099009D00A000A300A700AA00AE00B158
:103F400000B400B800BB00BF00C200C600C900CD6D
:103F500000D000D300D700DA00DE00E100E400E882
:103F600000EB00EF00F200F600F900FC0000010396
:103F70000107010A010E011101140118011B011FA3
:103F8000012201260129012C013001330137013AB8
:103F9000013D014101440148014B014E01520155CF
:103FA0000159015C016001630167016A016D0171E2
:103FB00001740178017B017E018201850189018CF8
:103FC000019001930196019A019D01A101A401A80C
:103FD00001AB01AE01B201B501B901BC01BF01C322
:103FE00001C601CA01CD01D101D401D801DB01DE36
:103FF00001E201E501E901EC01F001F301F601FA4A
:1040000001FD010102040208020B020E0212021558
:104010000219021C021F02230226022A022D02316B
:1040200002340237023B023E024202450249024C80
:10403000024F02530256025A025D02600264026796
:10404000026B026E027202750279027C027F0283A9
:104050000286028A028D029002940297029B029EBF
:1040600002A202A502A802AC02AF02B302B602B9D4
:1040700002BD02C002C402C702CB02CE02D102D5E9
:1040800002D802DC02DF02E302E602E902ED02F0FE
:1040900002F402F702FA02FE020103050308030C10
:1040A000030F031303160319031D0320032403271F
:1040B000032B032E033103350338033C033F034234
:1040C00003460349034D035003540357035A035E49
:1040D000036103650368036C036F0372037603795E
:1040E000037D038003840387038A038E0391039572
:1040F0000398039B039F03A203A603A903AD03B088
:1041000003B303B703BA03BE03C103C503C803CC9B
:1041100003CF03D203D603D903DC03E003E303E7B1
:1041200003EA03EE03F103F503F803FB03FF0300C7
:104130000000FC04FC07FC0AFC0EFC11FC15FC183A
:10414000FC1BFC1FFC22FC26FC29FC2DFC30FC3354
:10415000FC37FC3AFC3EFC41FC45FC48FC4BFC4F68
:10416000FC52FC56FC59FC5CFC60FC63FC67FC6A7E
:10417000FC6EFC71FC75FC78FC7BFC7FFC82FC8691
:10418000FC89FC8CFC90FC93FC97FC9AFC9EFCA1A7
:10419000FCA4FCA8FCABFCAFFCB2FCB6FCB9FCBCBC
:1041A000FCC0FCC3FCC7FCCAFCCDFCD1FCD4FCD8D1
:1041B000FCDBFCDFFCE2FCE5FCE9FCECFCF0FCF3E6
:1041C000FCF7FCFAFCFDFC01FD04FD08FD0BFD0FF6
:1041D000FD12FD15FD19FD1CFD20FD23FD26FD2A08
:1041E000FD2DFD31FD34FD38FD3BFD3EFD42FD451D
:1041F000FD49FD4CFD50FD53FD57FD5AFD5DFD6130
:10420000FD64FD68FD6BFD6EFD72FD75FD79FD7C45
:10421000FD80FD83FD86FD8AFD8DFD91FD94FD975A
:10422000FD9BFD9EFDA2FDA5FDA9FDACFDAFFDB36F
:10423000FDB6FDBAFDBDFDC1FDC4FDC7FDCBFDCE84
:10424000FDD2FDD5FDD9FDDCFDDFFDE3FDE6FDEA98
:10425000FDEDFDF1FDF4FDF7FDFBFDFEFD02FE05AC
:10426000FE08FE0CFE0FFE13FE16FE1AFE1DFE21BA
:10427000FE24FE27FE2BFE2EFE32FE35FE38FE3CCF
:10428000FE3FFE43FE46FE4AFE4DFE50FE54FE57E4
:10429000FE5BFE5EFE61FE65FE68FE6CFE6FFE73F9
:1042A000FE76FE79FE7DFE80FE84FE87FE8BFE8E0E
:1042B000FE91FE95FE98FE9CFE9FFEA3FEA6FEA923
:1042C000FEADFEB0FEB4FEB7FEBBFEBEFEC1FEC537
:1042D000FEC8FECCFECFFED2FED6FED9FEDDFEE04D
:1042E000FEE4FEE7FEEAFEEEFEF1FEF5FEF8FEFC61
:1042F000FEFFFE02FF06FF09FF0DFF10FF14FF1770
:10430000FF1AFF1EFF21FF25FF28FF2CFF2FFF3282
:10431000FF36FF39FF3DFF40FF43FF47FF4AFF4E97
:10432000FF51FF55FF58FF5BFF5FFF62FF66FF69AC
:10433000FF6DFF70FF73FF77FF7AFF7EFF81FF85C0
:10434000FF88FF8BFF8FFF92FF96FF99FF9DFFA0D5
:10435000FFA3FFA7FFAAFFAEFFB1FFB4FFB8FFBBEB
:10436000FFBFFFC2FFC6FFC9FFCCFFD0FFD3FFD7FF
:10437000FFDAFFDDFFE1FFE4FFE8FFEBFFEFFFF215
:10438000FFF6FFF9FFFCFF0000010104020602072F
:104390000209020B020C020E021002120213021595
:1043A00002170218021A021C021E021F0221022317
:1043B000022402260228022A022B022D022F02309A
:1043C00002320234023502370239023B023C023E1D
:1043D000024002410243024502470248024A024C9F
:1043E000024D024F02510253025402560258025922
:1043F000025B025D025F02600262026402650267A4
:104400000269026B026C026E027002710273027525
:1044100002760278027A027C027D027F02810282A9
:104420000284028602880289028B028D028E02902B
:1044300002920294029502970299029A029C029EAD
:1044400002A002A102A302A502A602A802AA02AC2F
:1044500002AD02AF02B102B202B402B602B802B9B2
:1044600002BB02BD02BE02C002C202C302C502C735
:1044700002C902CA02CC02CE02CF02D102D302D5B7
:1044800002D602D802DA02DB02DD02DF02E102E23A
:1044900002E402E602E702E902EB02ED02EE02F0BC
:1044A00002F202F302F502F702F802FA02FC02FE3F
:1044B00002FF02010303030503060308030A030BBB
:1044C000030D030F0310031203140316031703193C
:1044D000031B031C031E03200322032303250327BE
:1044E0000328032A032C032E032F03310333033441
:1044F00003360338033A033B033D033F03400342C3
:104500000344034603470349034B034C034E035044
:1045100003520353035503570358035A035C035DC7
:10452000035F036103630364036603680369036B4A
:10453000036D036F037003720374037503770379CC
:10454000037B037C037E038003810383038503874E
:104550000388038A038C038D038F039103920394D2
:10456000039603980399039B039D039F03A003A253
:1045700003A403A503A703A903AA03AC03AE03B0D6
:1045800003B103B303B503B603B803BA03BC03BD59
:1045900003BF03C103C203C403C603C803C903CBDB
:1045A00003CD03CE03D003D203D403D503D703D95D
:1045B00003DA03DC03DE03DF03E103E303E503E6E1
:1045C00003E803EA03EB03ED03EF03F103F203F463
:1045D00003F603F703F903FB03FD03FE03000400E6
:1045E0000100FF00FC02FC03FC05FC07FC09FC0ABF
:1045F000FC0CFC0EFC0FFC11FC13FC15FC16FC184B
:10460000FC1AFC1BFC1DFC1FFC21FC22FC24FC26CC
:10461000FC27FC29FC2BFC2DFC2EFC30FC32FC334F
:10462000FC35FC37FC38FC3AFC3CFC3EFC3FFC41D2
:10463000FC43FC44FC46FC48FC4AFC4BFC4DFC4F54
:10464000FC50FC52FC54FC56FC57FC59FC5BFC5CD7
:10465000FC5EFC60FC62FC63FC65FC67FC68FC6A59
:10466000FC6CFC6EFC6FFC71FC73FC74FC76FC78DB
:10467000FC79FC7BFC7DFC7FFC80FC82FC84FC855F
:10468000FC87FC89FC8BFC8CFC8EFC90FC91FC93E1
:10469000FC95FC97FC98FC9AFC9CFC9DFC9FFCA163
:1046A000FCA3FCA4FCA6FCA8FCA9FCABFCADFCAFE5
:1046B000FCB0FCB2FCB4FCB5FCB7FCB9FCBBFCBC68
:1046C000FCBEFCC0FCC1FCC3FCC5FCC7FCC8FCCAEA
:1046D000FCCCFCCDFCCFFCD1FCD2FCD4FCD6FCD86D
:1046E000FCD9FCDBFCDDFCDEFCE0FCE2FCE4FCE5F0
:1046F000FCE7FCE9FCEAFCECFCEEFCF0FCF1FCF372
:10470000FCF5FCF6FCF8FCFAFCFCFCFDFCFFFC01F3
:10471000FD02FD04FD06FD08FD09FD0BFD0DFD0E6E
:10472000FD10FD12FD13FD15FD17FD19FD1AFD1CF1
:10473000FD1EFD1FFD21FD23FD25FD26FD28FD2A73
:10474000FD2BFD2DFD2FFD31FD32FD34FD36FD37F6
:10475000FD39FD3BFD3DFD3EFD40FD42FD43FD4578
:10476000FD47FD48FD4AFD4CFD4EFD4FFD51FD53FB
:10477000FD54FD56FD58FD5AFD5BFD5DFD5FFD607E
:10478000FD62FD64FD66FD67FD69FD6BFD6CFD6E00
:10479000FD70FD72FD73FD75FD77FD78FD7AFD7C82
:1047A000FD7EFD7FFD81FD83FD84FD86FD88FD8A04
:1047B000FD8BFD8DFD8FFD90FD92FD94FD95FD9788
:1047C000FD99FD9BFD9CFD9EFDA0FDA1FDA3FDA50A
:1047D000FDA7FDA8FDAAFDACFDADFDAFFDB1FDB38C
:1047E000FDB4FDB6FDB8FDB9FDBBFDBDFDBFFDC00F
:1047F000FDC2FDC4FDC5FDC7FDC9FDCBFDCCFDCE91
:10480000FDD0FDD1FDD3FDD5FDD7FDD8FDDAFDDC12
:10481000FDDDFDDFFDE1FDE3FDE4FDE6FDE8FDE995
:10482000FDEBFDEDFDEEFDF0FDF2FDF4FDF5FDF718
:10483000FDF9FDFAFDFCFDFFFE4E414E494E495487
:1048400059494E46CDCCCC3D0AD7233C17B7D13879
:1048500077CC2B329595E6241FB14F0A00002041FA
:104860000000C84200401C4620BCBE4CCA1B0E5A69
:10487000AEC59D7400407A10F35A00A0724E18091C
:104880000010A5D4E80000E87648170000E40B54B7
:10489000020000CA9A3B000000E1F5050000809686
:1048A0009800000040420F000000A08601000000B8
:1048B000102700000000E803000000006400000072
:1048C00000000A00000000000100000000002C763B
:1048D000D888DC674F0823DFC1DFAE59E1B1B79656
:1048E000E5E3E453C63AE651997696E8E6C28426B3
:1048F000EB898C9B62ED407C6FFCEFBC9C9F40F28F
:10490000BAA56FA5F490055A2AF75C936B6CF9670A
:104910006DC11BFCE0E40D47FEF520E6B500D0EDCF
:10492000902E0300943577050080841E0800002037
:104930004E0A000000C80C333333330F986E1283D5
:104940001141EF8D2114893BE65516CFFEE6DB18A9
:10495000D1844B381BF77C1D901DA4BBE42420326E
:1049600084725E228100C9F124ECA1E53D27E75362
:104970000A5411241FBECFEFCDBFDFE3DEBF00E03E
:104980000CBF18BE19BE1ABE1BBE10E2A0E0B0E2FA
:10499000E8EBF2EC00E00BBF02C007900D92A63DE1
:1049A000B107D9F71BBE26E2A6EDB0E201C01D9209
:1049B000A733B207E1F719E4C2E7D9E400E006C083
:1049C00022970109FE010BBF0E941D59CE36D10767
:1049D00080E00807A9F70E94E0530C945A610C94F8
:1049E00000008FE10E94C828019729F488ED84BF58
:1049F00023E02093800008951F920F920FB60F922C
:104A0000112408B60F9218BE09B60F9219BE0BB644
:104A10000F921BBE8F939F93AF93BF93EF93FF9320
:104A20008091DA209091DB20A091DC20B091DD20F4
:104A30000196A11DB11D8093DA209093DB20A093F5
:104A4000DC20B093DD209FE0E0E8F1E0908BFF9167
:104A5000EF91BF91AF919F918F910F900BBE0F90EF
:104A600009BE0F9008BE0F900FBE0F901F901895B3
:104A70001F920F920FB60F92112408B60F9218BE14
:104A800009B60F9219BE8F939F93AF93BF938091F6
:104A9000D6209091D720A091D820B091D92001960E
:104AA000A11DB11D8093D6209093D720A093D8202C
:104AB000B093D920BF91AF919F918F910F9009BE74
:104AC0000F9008BE0F900FBE0F901F901895CF92B9
:104AD000DF92EF92FF928FB7F8942091D620309119
:104AE000D7204091D8205091D920E0E4F9E000A0EF
:104AF000F1A1E02D8FBFC090DA20D090DB20E090B4
:104B0000DC20F090DD20A8EEB3E00E94DF586E0FAD
:104B10007F1F811D911D6C0D7D1D8E1D9F1DFF90A2
:104B2000EF90DF90CF9008952F923F924F925F9237
:104B30006F927F928F929F92AF92BF92CF92DF92AD
:104B4000EF92FF920F931F932FB7F8946091D620A6
:104B50007091D7208091D8209091D920E0E4F9E09D
:104B600080A091A0E0E0F9E0A0A0B1A02FBFB69492
:104B7000A794B694A79420E432E44FE050E00E945A
:104B8000F25829013A01B62FA72FF82F292E9501A7
:104B900040E050E060E070E080E090E052016301AE
:104BA000EB2EFA2E0F2F122D0E94225979018B0124
:104BB000782EB92E9401A8EEB3E00E94C9581B01CB
:104BC0002C019701B801872D9B2D51016201E12C29
:104BD000F12C00E010E00E9422591F910F91FF90EC
:104BE000EF90DF90CF90BF90AF909F908F907F908D
:104BF0006F905F904F903F902F9008958F929F926B
:104C0000AF92BF92CF92DF92EF92FF92CF93DF935A
:104C10008FB7F8948090DA209090DB20A090DC2071
:104C2000B090DD202091D6203091D7204091D8201F
:104C30005091D920E0E0F9E000A0F1A1E02DA0E43E
:104C4000B9E09096CD91DC9191978FBFF695E7955D
:104C5000F695E79560E472E48FE090E00E946A5870
:104C60006B017C01CE0EDF1EE11CF11C8C0E9D1E23
:104C7000A11CB11CA8EEB3E0A50194010E94DF586D
:104C8000C60ED71EE81EF91EC701B601DF91CF91EF
:104C9000FF90EF90DF90CF90BF90AF909F908F905C
:104CA00008958F929F92AF92BF92CF92DF92EF9230
:104CB000FF926C010E94FE254B015C01E12CF12C5E
:104CC0000E94FE25681979098A099B09C616D7062C
:104CD000E806F906A8F7FF90EF90DF90CF90BF901D
:104CE000AF909F908F9008958F929F92AF92BF92B6
:104CF000CF92DF92EF92FF926B017C010E946725B9
:104D00004B015C010E946725681979098A099B0992
:104D1000C616D706E806F906A8F7FF90EF90DF90D1
:104D2000CF90BF90AF909F908F900895789480E13E
:104D300080935500209150002061209350003091C5
:104D4000510034FFFCCF48ED44BF50914000587FE4
:104D500054605093400062E160936D007AE7709375
:104D60006E00A1E0A093680094E090930009E0EA4F
:104D7000FFE0E0933609F0933709B0910109B87F5D
:104D8000B0930109F2E0F093060988E080934009AE
:104D900028EE33E02093760930937709309141096A
:104DA000387F3093410940E540934309F093460929
:104DB00057E8509387016FEF6093B00070E17093F4
:104DC00010061092000610920102709302021092D7
:104DD000030296E09093040210920602A093200230
:104DE00010922202A0932302A09300026093B000CD
:104DF00070933006109220066093B0001092500617
:104E00006093B000109270066093B000109290060C
:104E100042E050E061EF74E28FE10E944429A091EA
:104E2000A200A760A093A200789408958093002028
:104E300008958C3028F5E82FF0E0EC53FA4F859177
:104E40009491909100209295907F9093020220E19E
:104E500020930102880F880F880F80932102809190
:104E600020028068809320023091230230FFFCCF23
:104E700041E0409323028091100290911102089525
:104E80008FEF9FEF08950E94192797FF02C080E0DF
:104E900090E09595879508950E941927BC01882771
:104EA00077FD8095982F3CE0660F771F881F991F2C
:104EB0003A95D1F708950E94192744E0880F991F69
:104EC0004A95E1F708950E941927BC01882777FDCC
:104ED0008095982F0E94865521E038E040E859E3FC
:104EE0000E943A5608957F928F929F92AF92BF92FE
:104EF000CF92DF92EF92FF920F931F93CF93DF93A6
:104F0000782E5B01E82FF0E0EB5DF94F8491282FBC
:104F100030E0220F331FF901ED5FF94F0591149135
:104F2000F901EF51FA4FC591D491E82FF0E0E05329
:104F3000FA4FC590D4902E553A4FF901E590F49070
:104F400061E0872D0E94FA2701151105A1F04FEFAE
:104F500050E0E8014EAB5FAB55E058836981676074
:104F60006983D98020E130E001C0220FCA94EAF7BA
:104F7000D22AD98214C0209791F02FEF30E02EABC7
:104F80003FAB15E01883398137603983998020E180
:104F900030E001C0220FCA94EAF7922A9982E11404
:104FA000F10489F0F701A082B182DF91CF911F91C6
:104FB0000F91FF90EF90DF90CF90BF90AF909F90B8
:104FC0008F907F900895F0E8AF16B10414F460E07C
:104FD00001C061E0872DDF91CF911F910F91FF906C
:104FE000EF90DF90CF90BF90AF909F908F907F9089
:104FF0000C944A28EF92FF921F93CF93DF931F9256
:10500000CDB7DEB7E82EF12CF701E95BF94F14912B
:10501000812F69830E942429F701E759F94FE49110
:105020006981EE2381F1F0E0EE0FFF1FE557F94FA4
:10503000A591B491AD01405F5F4F9FB7F894282FC1
:1050400030E0611103C012961C9316C0633041F426
:1050500012961C93FA01E20FF31F8081806111C048
:10506000623041F412961C93FA01E20FF31F808123
:10507000886107C011961C93FA01E20FF31F80812B
:10508000877C80839FBF0F90DF91CF911F91FF900E
:10509000EF900895CF92DF92EF92FF921F93CF93FC
:1050A000DF931F92CDB7DEB7E82EF12CF701E95B55
:1050B000F94F1491812F69830E942429F701EB5D38
:1050C000F94F7491F701E759F94F94916981992348
:1050D00009F455C0772391F1272F30E0220F331FB9
:1050E000F901ED5FF94FC590D4902F513A4FF90176
:1050F000A591B491E72FF0E0E053FA4FE590F490DA
:10510000C114D10461F0F601F18020E130E001C06A
:10511000220FEA94EAF720952F2121830FC01097E0
:1051200069F01196DC90119720E130E001C0220F68
:10513000EA94EAF720952D2111962C93E92FF0E0BF
:10514000EE0FFF1FE557F94FA591B4912FB7F894D3
:10515000EC90E12261F4509690E0A80FB91F8C9179
:10516000611102C0877E01C088618C9307C0611104
:1051700003C016961C9302C015961C932FBF0F9068
:10518000DF91CF911F91FF90EF90DF90CF90089526
:105190000F931F93CF93DF9390E0FC01EB5DF94FEA
:1051A0004491FC01E95BF94F6491FC01E759F94F27
:1051B0008491882309F441C0442381F1242F30E0F5
:1051C000220F331FF901ED5FF94FC591D4912F5193
:1051D0003A4FF901A591B491E42FF0E0E053FA4F72
:1051E00045915491209759F0198120E130E001C098
:1051F000220F4A95EAF72095212329830FC01097A3
:1052000069F011969C91119720E130E001C0220FC6
:105210004A95EAF72095292311962C93E82FF0E080
:10522000EE0FFF1FE557F94FC591D491288526232E
:1052300081E090E021F480E002C080E090E0DF9126
:10524000CF911F910F9108958031A1F038F48430EF
:1052500069F0883069F0823039F414C0803471F01C
:10526000803871F0803241F080E0089582E0089546
:1052700083E0089584E0089585E0089586E0089528
:1052800087E0089581E00895AF92BF92CF92DF92B8
:10529000EF92FF920F931F93CF93DF936B018033B5
:1052A00008F04BC04530510540F4FA01EA57FF4D74
:1052B0000081112707FD109502C000E010E090E08A
:1052C0009C012759394F5901F9011491212F30E0E0
:1052D000220F331F2557394FF901C591D491AC01E5
:1052E000495B594F7A01FA0184910E942429F50102
:1052F000A491B0E0119753E0AA0FBB1F5A95E1F7B4
:10530000A80FB11DAA0FBB1FAC51BF4DCD92DC92AF
:10531000998594609987BB84F701C490CB28CB868C
:10532000FE017096E80FF11D8081802B8083D88468
:10533000E12FF0E0E252FF4DD082DF91CF911F913B
:105340000F91FF90EF90DF90CF90BF90AF900895B6
:10535000CF92DF92EF92FF920F931F93CF93DF9341
:10536000803308F03EC0082F10E0C8018759994FDC
:105370007C01FC01249130E0220F331F2557394F67
:10538000F901C591D4916E01F0E1CF0ED11C095BFA
:10539000194FF80184910E942429F701A491B0E0EB
:1053A0001197E3E0AA0FBB1FEA95E1F7A80FB11D23
:1053B000AA0FBB1FAC51BF4D1D921C929B85F801DB
:1053C0000491009509230B87FB84E82FF0E0F1108E
:1053D00003C01985137F1987EC0DFD1D2081287FDF
:1053E0002083DF91CF911F910F91FF90EF90DF907D
:1053F000CF9008956F927F929F92AF92BF92CF927B
:10540000DF92EF92FF920F931F93CF93DF93FC01F4
:10541000EE0FFF1FE557F94FC591D491D884FC01D9
:10542000E252FF4DC0800197A82EAA0CAA0CAA0C2C
:10543000D0828E01005F1F4FB12C992493942B2DA5
:105440002A0D3D2D3170632F692570E08C2D817000
:10545000A82FA925B0E0882311F03B0102C0612CE0
:10546000712C109741F091E0E12C311101C090E0D6
:10547000492F5E2D02C040E050E0F80181918F017C
:10548000877030E0220F331FF901EC51FF4DE080AF
:10549000F180EF28A1F0811104C0A617B70731F5FC
:1054A0000EC0813019F4452B09F509C0823019F47A
:1054B0006728E1F404C0833011F4672BB9F4D69463
:1054C000C694B394F8E0BF12BACF1C851D7F1C8729
:1054D000DF91CF911F910F91FF90EF90DF90CF90D0
:1054E000BF90AF909F907F906F900895F901EC511D
:1054F000FF4D0190F081E02D1995E1CF1F920F92A1
:105500000FB60F92112408B60F9218BE09B60F926B
:1055100019BE0BB60F921BBE2F933F934F935F9311
:105520006F937F938F939F93AF93BF93EF93FF936B
:1055300081E090E00E94FA29FF91EF91BF91AF9135
:105540009F918F917F916F915F914F913F912F919B
:105550000F900BBE0F9009BE0F9008BE0F900FBEAC
:105560000F901F9018951F920F920FB60F92112453
:1055700008B60F9218BE09B60F9219BE0BB60F925D
:105580001BBE2F933F934F935F936F937F938F93A4
:105590009F93AF93BF93EF93FF9382E090E00E94BD
:1055A000FA29FF91EF91BF91AF919F918F917F91D8
:1055B0006F915F914F913F912F910F900BBE0F9084
:1055C00009BE0F9008BE0F900FBE0F901F90189548
:1055D0001F920F920FB60F92112408B60F9218BEA9
:1055E00009B60F9219BE0BB60F921BBE2F933F93B5
:1055F0004F935F936F937F938F939F93AF93BF93DB
:10560000EF93FF9383E090E00E94FA29FF91EF91DE
:10561000BF91AF919F918F917F916F915F914F91CA
:105620003F912F910F900BBE0F9009BE0F9008BEB7
:105630000F900FBE0F901F9018951F920F920FB6EC
:105640000F92112408B60F9218BE09B60F9219BE18
:105650000BB60F921BBE2F933F934F935F936F93A5
:105660007F938F939F93AF93BF93EF93FF9384E0C8
:1056700090E00E94FA29FF91EF91BF91AF919F9125
:105680008F917F916F915F914F913F912F910F90EB
:105690000BBE0F9009BE0F9008BE0F900FBE0F906B
:1056A0001F9018951F920F920FB60F92112408B6F3
:1056B0000F9218BE09B60F9219BE0BB60F921BBE01
:1056C0002F933F934F935F936F937F938F939F930A
:1056D000AF93BF93EF93FF9385E090E00E94FA2988
:1056E000FF91EF91BF91AF919F918F917F916F91BA
:1056F0005F914F913F912F910F900BBE0F9009BE7C
:105700000F9008BE0F900FBE0F901F9018950E942B
:10571000443180E00C942233E82FF0E0E659FE4D4E
:105720006083E0917E2180E3E89FF0011124E95B32
:10573000FD4DA62FB0E0AA0FBB1FAC59BF4D2D9158
:105740003C912387348710A611A612A613A61682B1
:105750001782108611860895CF93DF9380917E2162
:1057600081110DC080918C2190E00E94903980932E
:1057700077219093782135E0309381210CC080917E
:105780008B2190E00E949039809374219093752131
:1057900024E120938021C0917E21D0E080918A2154
:1057A00090E00E949039FE01EE0FFF1FE459FE4D7C
:1057B0008083918345E040930120DF91CF9108954C
:1057C0000F931F93CF93DF9300917D2110E0C09141
:1057D0007E21D0E08091892190E00E949039F801EB
:1057E000EE0FFF1FEC0FFD1FEE0FFF1FE05BFE4DE6
:1057F0008083918300917D2110E0C0917E21D0E0D3
:105800008091882190E00E949039F801EE0FFF1FEF
:10581000EC0FFD1FEE0FFF1FEC5BFE4D80839183AD
:1058200085E08093832180938221DF91CF911F9126
:105830000F91089580E00E9442398823F9F081E0B9
:1058400090917F21911180E080937F21882371F0D6
:105850006091762180E00E94473A6091762181E054
:105860000E94473A21E020933D2208C080E00E9438
:105870006E3A81E00E946E3A10923D2281E00E94D1
:1058800042398823B9F030917E213F5F323019F0E0
:1058900030937E2102C010927E2140917E214130C2
:1058A00019F440933E2202C010923E220E94AC2B7B
:1058B0000E94E02B82E00E944239882391F05091AF
:1058C0007D21513031F061E060937D2160933F2272
:1058D00004C010927D2110923F22109240220E941B
:1058E000E02B83E00E9442398823A9F070917D214A
:1058F000723049F0A2E0A0937D2110923F22B1E0E6
:10590000B093402206C010927D2110923F22109247
:1059100040220C94E02B08952F923F924F925F9279
:105920006F927F928F929F92AF92BF92CF92DF92AF
:10593000EF92FF920F931F93CF93DF93CDB7DEB714
:105940002A97CDBFDEBF0E9469355DE2A52E52E2E7
:10595000B52E0DE312E2F50180819181A281B38120
:10596000892B8A2B8B2BC1F00E946725D501CD9006
:10597000DD90ED90FC906C157D058E059F0560F027
:1059800021E0F8019081911120E0D8012C93F501DC
:105990001082118212821382F4E0AF0EB11C0F5FED
:1059A0001F4F2DE3A21622E2B206A9F60E941A2C7E
:1059B00020907F21222009F442C030907E213110B6
:1059C0003EC080918C2190E00E949039BC014090B3
:1059D0007721509078213C016418750877FE03C048
:1059E0007194619471088091812190E086159705EA
:1059F00034F56093772170937821882777FD80951F
:105A0000982F1F921F921F922DE32F9335E1A32E03
:105A1000B12CC12CD12CE12C14E0F12E00E010E0CF
:105A200020E030E0A9010E94444160937621609318
:105A30004722609377220F900F900F900F90109154
:105A40007E21113009F07AC080918B2190E00E9474
:105A500090394C01E0907421F0907521AC014E1901
:105A60005F09BA0157FF03C07195619571094091B3
:105A7000802150E0461757070CF060C032E03093A9
:105A80008021809274219092752184010E561140DC
:105A9000073C110508F447C0B401882777FD8095BD
:105AA000982F5EE6851651E09506C4F41F921F926A
:105AB0001F921F92A12C14E0B12EC12CD12C1DE6F7
:105AC000E12EFF24F39400E010E020E030E0A90193
:105AD0000E94444171956195710914C01F921F92F3
:105AE00054E05F931F92A12CB12C6501EE24EA943F
:105AF00013E0F12E00E010E025E332E040E050E05A
:105B00000E9444410F900F900F900F90882777FDCF
:105B10008095982F0E94865520E030E040E85AE3B7
:105B20000E943A5603C060E070E0CB0160937021A0
:105B300070937121809372219093732180918721BA
:105B400090E00E949039BC01882777FD8095982FBE
:105B50001F921F921F92E0E49E2E9F92A12CB12CC7
:105B60006501EE24EA9413E0F12E00E010E020E05D
:105B700030E0A9010E944441609368218091862110
:105B800090E00E949039BC01882777FD8095982F7E
:105B90001F921F921F929F9220E030E0A9010E9465
:105BA00044416093692180918A2190E00E9490395C
:105BB0001C01E0917E21F0E0EE0FFF1FE459FE4D45
:105BC000A080B1802C014A185B0857FE03C0519495
:105BD000419451081F921F921F927CE07F93A12C49
:105BE000B12C6501E12C14E0F12E00E010E020E082
:105BF00030E0A901B101882777FD8095982F0E9498
:105C000044412091012030E0CDBFDEBF2415350591
:105C1000C4F450907E21E52DF0E0DF01A659BE4D81
:105C20002C9130E02617370761F0B2E0B0930120E5
:105C3000EE0FFF1FE459FE4D20823182852D0E9418
:105C40008C2B8091852190E00E94903995958795C5
:105C5000959587958093792190937A21709064210E
:105C6000711007C0809334239093352380E00E9405
:105C70006D3B8091842190E00E94903995958795A5
:105C80009595879580937B2190937C21B090652199
:105C9000B11007C0809336239093372381E00E9490
:105CA0006D3B8091892190E00E9490394C011C014C
:105CB000442437FC4094542C1F921F92F3E0FF932E
:105CC0008FEF8F93A12CB12C6501EE24EA9413E0A1
:105CD000F12E00E010E025E030E040E050E0C201AD
:105CE000B1010E94444100917D2110E0E0907E21AD
:105CF000F12C000F111FF801EE0DFF1DEE0FFF1F1D
:105D0000E05BFE4DC080D18094012C193D09390122
:105D100037FF03C07194619471082091832130E0B2
:105D20000F900F900F900F90261537050CF074C050
:105D300010928321F801EE0DFF1DAF01440F551F96
:105D4000DA01A05BBE4D8D929C92EE59FE4D181467
:105D500019040CF045C0D080D11005C0FA01E553FC
:105D6000FD4D10821182C8018E0D9F1DFC01EE5960
:105D7000FE4D61E06083880F991F880F991F811481
:105D8000F2E09F0674F4865F9C4D6C01C201B10184
:105D90000E94865528E230E540E25CE30E943A56D4
:105DA00018C0FC01E65FFC4D6F01B40172508827FA
:105DB00077FD8095982F0E9486552EEC31EE45E4B4
:105DC0005FE30E943A5620E030E040EA50E40E944F
:105DD000EB54D6016D937D938D939C93139701C0E3
:105DE00010820E0D1F1DF801EE0FFF1FEE0FFF1F9B
:105DF000EE50FD4D20E030E0A9016081718182818B
:105E000093810E944F55811107C0F801EE0FFF1FCB
:105E1000EC5BFE4D108211828091882190E00E94FF
:105E200090394C01BC01882777FD8095982F1F92EF
:105E30001F9213E01F933FEF3F9324E1A22EB12C5A
:105E4000C12CD12CEE24EA9413E0F12E00E010E0F6
:105E500020E030E0A9010E94444120917D2130E002
:105E6000A0917E21B0E0220F331FF901EA0FFB1F42
:105E7000EE0FFF1FEC5BFE4DE080F1808E189F0857
:105E800097FE03C09194819491084091822150E043
:105E90000F900F900F900F9048155905E4F4109251
:105EA00082218D01020F131F000F111F000F111F00
:105EB0000E501D4D882777FD8095982F0E9486559E
:105EC00028E030E240E85AE30E943A56F801608345
:105ED000718382839383B3E6AB2EB1E2BB2E00E0E5
:105EE000F5013197F080FF2021F060E0802F0E94C3
:105EF000A239D5019C91992321F061E0802F0E9465
:105F0000A2390F5FB2E0AB0EB11C033049F73090FD
:105F1000622130925C215091642150935E219090D7
:105F20006621909260214090632140925D217091A2
:105F3000652170935F21509067215092612128E67E
:105F400032E22F83388748E651E24D835E8369E76A
:105F500071E26B837C83EAED4E2EE2E25E2EF2EF7D
:105F60002F2EF2E23F2E84E393E289839A8300E0AE
:105F700010E0A0E36A2E702E609EF001619EF00D8D
:105F80001124E95BFD4DE987FA87B081B23008F44E
:105F900030C1B080F4E0BF9EF0011124E75CFE4DFB
:105FA000C080D180E280F380E985FA85C282D38205
:105FB000E482F58231E003136DC0C0907021D0906F
:105FC0007121E0907221F090732120E030E0A9016E
:105FD000C701B6010E944F55882309F45BC0A9850B
:105FE000BA8512968D909D90AD90BC90159720E04B
:105FF00030E0A901C701B6010E944F5587FF17C0C5
:10600000E985FA85808190E046971CF07081715097
:1060100001C075E124E0729FF0011124E75CFE4DA0
:106020002081318142815381C501B40117C0E985C6
:10603000FA85208130E02C3331051CF490819F5F7C
:1060400001C09CE354E0959FF0011124E75CFE4DF4
:10605000A501940160817181828193810E94EA543B
:10606000A70196010E943A56609E7001619EF00C55
:106070001124F701E95BFD4D5F01228133814481E9
:1060800055810E94EB54D50112966D937D938D93AB
:106090009C931597F801EE59FE4D5F01D080DD20ED
:1060A00099F1609EA001619E500D1124BA01695BB7
:1060B0007D4D4B01DB0112966D917D918D919C91EF
:1060C00015971296CD90DD90ED90FC90159720E0FD
:1060D00030E040E05FE30E943A56F20120813181D6
:1060E000428153810E943A56D1012D913D914D91AB
:1060F0005C910E943A56A70196010E94EB54F4016C
:106100006283738384839583D5011296FC90FF206C
:1061100041F1F1012085318542855385D2011896E0
:106120006D917D918D919C911B970E943A5620E034
:1061300030E040E852E40E943A560E945355EB8109
:10614000FC8120813181260F371F2F3F310519F047
:1061500014F02FEF30E0C90137FF0DC080E090E070
:106160000AC0F801E45AFE4D9280992059F0EB8163
:10617000FC8180819181A981BA818D939C93872D27
:106180000E946D3BF501B480AD81BE81BB2031F131
:10619000EC90F12CF1012089318942895389D20197
:1061A00050966D917D918D919C9153970E943A5696
:1061B00020E030E040E852E40E943A560E945355F5
:1061C0006E0D7F1D77FD06C0613471052CF060E413
:1061D00070E002C060E070E0FB0102C0EC91F0E012
:1061E000EE5FFF4DB081EF81F885B083872D0E946F
:1061F000893A0F5F1F4F4F815885405D5F4F4F8336
:1062000058876D817E816F5F7F4F6D837E838B8129
:106210009C8102968B839C8394E0490E511CA4E0E0
:106220002A0E311CA981BA811296A983BA83023041
:10623000110509F0A0CE03E410E27DE3472E72E2DF
:10624000572EF20161912F01F80181918F010E9477
:106250004A28F1E44F16F2E25F0699F72A96CDBF7D
:10626000DEBFDF91CF911F910F91FF90EF90DF90F4
:10627000CF90BF90AF909F908F907F906F905F90E6
:106280004F903F902F900895CF93DF9362E08CE082
:106290000E94FA2762E08DE00E94FA2762E08FE018
:1062A0000E94FA2762E08EE00E94FA2761E088E10E
:1062B0000E94FA2761E089E10E94FA2761E084E107
:1062C0000E94FA2761E085E10E94FA2783E00E949C
:1062D000162785E080932003109221031092220359
:1062E000C0E0D0E0C0933803D09339038AE090E057
:1062F0000E9451262196C11588E0D80799F721E020
:1063000020930008109201081092020810920308CE
:106310001092040840E055E0409326085093270867
:1063200033E0309306082093400810924108109201
:106330004208109243081092440860E07DE76093A1
:1063400066087093670820934608DF91CF910895FF
:106350000F931F93CF93DF93082FEB01682F80E0FB
:106360000E94223A11E01093512220916620309130
:1063700067202093522230935322602F70E065549F
:106380007109882777FD8095982F0E9486552BEA02
:106390003AEA4AEA5DE30E943A569B01AC0160E0AA
:1063A00070E080E090E40E949D5620E030E04CEDEB
:1063B00053E40E943A566093492270934A22809394
:1063C0004B2290934C2280E4809367228093682232
:1063D00080E00E94893ABE01882777FD8095982F3A
:1063E0000E94742610934722DF91CF911F910F9145
:1063F0000895BC0181E50C94A831AF92BF92CF9271
:10640000DF92EF92FF920F931F93CF93DF9382E37C
:1064100090E00E94F93169E170E080E090E00E9434
:10642000742682E390E00E94F93168EC70E080E02D
:1064300090E00E94742665E480E00E94223A80E0A9
:1064400090E0ACEDB3E48093492290934A22A0936C
:106450004B22B0934C2280E00E94893A00E40093E2
:10646000672200936822C1E0DFEF83E00E943F399A
:10647000882309F466C087E090E00E949039BC014F
:10648000882777FD8095982F1F921F92CF93DF93D7
:10649000A12C2EEFB22ECC24CA94DC2CEE24EA944C
:1064A00013E0F12E00E010E020E030E0A9010E94AE
:1064B00044416093412270934222882777FD809562
:1064C000982F0E94865520E030E040E85BE30E9470
:1064D0003A5620E030E040E05FE30E94EA546093E7
:1064E00056207093572080935820909359202BEA80
:1064F0003AEA4AEA5DE30E943A569B01AC0160E049
:1065000070E080E090E40E949D5620E030E04CED89
:1065100053E40E943A566093492270934A22809332
:106520004B2290934C2280E00E94893A6AE070E00E
:1065300080E090E00E9474260F900F900F900F90D3
:1065400094CF11E010934722DF91CF911F910F91CB
:10655000FF90EF90DF90CF90BF90AF900C943E38BB
:106560008F929F92AF92BF92CF92DF92EF92FF9263
:106570000F931F93CF93DF93C82F813021F482E3D1
:1065800090E00E94F93199249394C13009F4912C40
:1065900000E054E0852E892D0E943F398823A1F127
:1065A00084E090E00E949039BC01882777FD8095B7
:1065B000982F1F921F921F928F92A12CB12C6501D0
:1065C000E12C14E0F12E00E010E020E030E0A90121
:1065D0000E944441062FC3E4D0E20F900F900F9029
:1065E0000F9010E0101307C0E12FF0E0ED5BFF4DBE
:1065F00061E0808102C060E088810E944A281F5FBC
:106600002196143079F7C7CF64E170E080E090E024
:106610000E947426C3E4D0E260E089910E944A2877
:1066200080E2C734D807C1F7802FDF91CF911F9147
:106630000F91FF90EF90DF90CF90BF90AF909F9021
:106640008F9008954F925F926F927F928F929F9258
:10665000AF92BF92CF92DF92EF92FF920F931F9370
:10666000CF93DF93182FEBE4F0E287E490E2CDE3E1
:10667000D2E24DE252E221E02193DC012D93CD01E3
:106680001992DA011D921D921D921D92AD01B0E288
:10669000EF34FB0789F780E00E946E3A81E00E94A8
:1066A0006E3A4090642050906520A2E6B2E20DE47C
:1066B000E02E02E2F02E20E030E070E36FEF729FF8
:1066C000F001739FF00D1124E95BFD4D1082CD01A7
:1066D0000197EC0118826C93128213821482158246
:1066E000E701188219821A821B824097EC011882F6
:1066F000E7014D825E820396EC0118820196EC015F
:10670000188210A611A612A613A614A615A62F5F0E
:106710003F4FD096D0E3ED0EF11C2230310579F6D3
:1067200010927F214FEF50E0409334235093352354
:10673000409336235093372340933223509333238F
:1067400080E00E946D3B81E00E946D3B111105C00D
:1067500080E00E943F39811199C181E00E943F3958
:106760008823C9F080E00E94B032809355200E94B7
:106770008736811110C064E670E08DE20E94A83176
:1067800064E670E080E090E00E94742664E670E0C9
:106790008DE20E94A8310E94283883E00E943F3990
:1067A000882319F0112309F480C16091412270916E
:1067B0004222882777FD8095982F0E94865520E0F9
:1067C00030E040E85BE30E943A5620E030E040E0F1
:1067D0005FE30E94EA546B017C0160935620709342
:1067E000572080935820909359200DE811E2C0ED76
:1067F000DFEFBE01882777FD8095982F0E94865590
:10680000A70196010E94EB542BEA3AEA4AEA5DE3BB
:106810000E943A569B01AC0160E070E080E090E499
:106820000E949D5620E030E04CED53E40E943A5621
:10683000F80161937193819391938F012196C83FE1
:10684000FFEFDF07B1F610928C2110928B2101E04F
:1068500000938A2132E03093892153E050938821BC
:1068600094E090938721B6E0B0938621D5E0D09351
:106870008521F7E0F093842120E531E2C4E4D1E200
:10688000AAE0B3E212EF612E12E2712E40E050E076
:1068900080E090E0BA016E597E4D6B01FB011082E1
:1068A0008A01045A1E4D2801F8011082F901108254
:1068B0001182188219821D921D921D921C921397AB
:1068C000F30110821182128213824C01880C991CF0
:1068D000880C991C840105531D4DF801108211820A
:1068E000F401E154FD4D5F0110821182BC01660F7D
:1068F000771FFB01E754FD4D7F0110826D547D4DE4
:10690000FB011082F6011182F2011182F90112825B
:1069100013821A821B8214961D921D921D921C9244
:106920001797F3011482158216821782F8011282DA
:106930001382F50112821382F7011182FB01118289
:1069400001964E5F5F4F2C5F3F4F24961896F8E0FC
:106950006F0E711C8330910509F09CCF10927E213F
:1069600010927D211092702110927121109272214B
:106970001092732181E090E00E94903980936C2105
:1069800090936D2180936E2190936F213C01882418
:1069900077FC8094982C1F921F921F92DCE0DF936B
:1069A000A12CB12C6501E12C14E0F12E00E010E0E7
:1069B00020E030E0A901C401B3010E94444160938A
:1069C0006A211F921F921F92DF9320E030E0A901FD
:1069D000C401B3010E94444160936B2180918B21DB
:1069E00090E00E949039809374219093752180915A
:1069F0008C2190E00E9490398093772190937821A8
:106A00001F921F921F927DE37F9375E1A72EB12CF9
:106A1000C12CD12C20E030E0A901C401B3010E94B7
:106A2000444160937621809155202DB73EB7245F75
:106A30003F4F2DBF3EBF8F3F31F00E9475370E9400
:106A4000AC2B0E94E02B0E943E3862E370E080E0B5
:106A500090E00E947426C3E4D0E261E089910E9434
:106A60004A2830E2C734D307C1F768EC70E080E011
:106A700090E00E947426C3E4D0E260E089910E9415
:106A80004A2860E2C734D607C1F712C081E00E94ED
:106A90003F39882339F00E94553882E390E00E9404
:106AA000F93179CE0E941E3676CE0E94FD317DCE20
:106AB000DF91CF911F910F91FF90EF90DF90CF90DA
:106AC000BF90AF909F908F907F906F905F904F900E
:106AD00008950F931F938EE00E94C82821E0892B10
:106AE00009F020E08091B122281799F0222371F05B
:106AF0000E9467256093AD227093AE228093AF22EF
:106B00009093B02231E03093B12239C01092B1227B
:106B100036C02223A1F10E9467250091AD22109179
:106B2000AE222091AF223091B022601B710B820BFC
:106B3000930B613D77408105910508F11092B122D8
:106B40001FEF1093552080E00E943F39882391F079
:106B500080E00E946E3A81E00E946E3A81E00E94DD
:106B6000B032809355200E94AA3662E370E081E53E
:106B70000E94A83181E01F910F910C9422331F9144
:106B80000F910895CF93C82F80914722811113C090
:106B90006C2F0E94223A81E080935122209166203E
:106BA00030916720209352223093532230E4309367
:106BB0006722309368226C2F70E065547109882732
:106BC00077FD8095982F0E9486552BEA3AEA4AEA8B
:106BD0005DE30E943A569B01AC0160E070E080E00A
:106BE00090E40E949D5620E030E04CED53E40E947A
:106BF0003A566093492270934A2280934B22909395
:106C00004C2280E0CF910C94893A0F931F93CF933D
:106C1000DF93C0E0D0E000E010E0CE010E949039A8
:106C2000081719070CF48C012196C830D105A9F773
:106C3000C801DF91CF911F910F91089549E4842EEF
:106C4000992493940E940536BC01882777FD80958E
:106C5000982F1F921F921F928F9220E3A22EB12C89
:106C6000C12CD12CE12C14E0F12E00E010E020E04A
:106C700030E0A9010E944441E62E10923D2210927C
:106C80003E2210923F221092402280E00E943F3923
:106C90000F900F900F900F90882329F090923D2233
:106CA000FF24F39401C0F12C81E00E943F39882336
:106CB00021F090923E22FF24F39482E00E943F391B
:106CC000882321F090923F22FF24F39483E00E94D6
:106CD0003F39882321F090924022FF24F394CDE3A2
:106CE000D2E203E410E26991F80181918F010E94E0
:106CF0004A28F2E2C134DF07B1F7FF2021F08E2DE0
:106D00000E94C2359FCF80E00E946E3A9BCFF894DC
:106D10002FE3829FC001112405960E94395D78946B
:106D200041E08B3A934E09F040E0842F0895909112
:106D3000B222913019F41092B22203C021E02093C4
:106D4000B222E82FF0E0ED5BFF4D6091B22280812E
:106D50000C944A282F923F924F925F926F927F92AB
:106D60008F929F92AF92BF92CF92DF92EF92FF925B
:106D70000F931F93CF93DF9300D01F92CDB7DEB751
:106D8000082F882E912CB4018BE890E20E94C6381F
:106D9000F8948FE3089F10011124210195E0490E1A
:106DA000511C6BEA73EEC2010E94695D609176210D
:106DB000C10107960E943E5D409170215091712162
:106DC0006091722170917321C10108960E94615DEA
:106DD00060916A21C1010C960E943E5D60916B2119
:106DE000C1010D960E943E5D5101AEE0AA0EB11C9C
:106DF00082E6682E81E2782E00E010E09501E12C19
:106E0000F12CC12CD12CD801A65FBC4D1D01F8017D
:106E1000EE50FD4DE983FA83F301EC0DFD1D608119
:106E2000C9012B833C830E943E5DF101EE0DFF1DE5
:106E300040815181628173812B813C81C90101961E
:106E40000E94615DE981FA81EE0DFF1D4081518153
:106E5000628173812B813C81C90105960E94615D2D
:106E60002B813C81275F3F4FBFEFCB1ADB0AE4E069
:106E7000EE0EF11CF2E0CF16D10471F682E1A80EFD
:106E8000B11C92E0690E711C085F1F4F083111059B
:106E900009F0B4CFF401ED5BFF4D60E080810E940A
:106EA0004A286FE370E089E990E20E94C638B20197
:106EB000615C7F4F81EA90E20E94C6387894249604
:106EC000CDBFDEBFDF91CF911F910F91FF90EF906B
:106ED000DF90CF90BF90AF909F908F907F906F90FA
:106EE0005F904F903F902F9008952F923F924F9236
:106EF0005F926F927F928F929F92AF92BF92CF924A
:106F0000DF92EF92FF920F931F93CF93DF93682E40
:106F1000882E912CB40180EB90E20E94C638862D19
:106F20000E948736882309F475C0F8948FE3689E21
:106F300030011124C30107960E94225D80937621BF
:106F4000C30108960E94325D609370217093712195
:106F50008093722190937321C3010C960E94225D4D
:106F600080936A21C3010D960E94225D80936B215C
:106F70009EE0690E711C92E6A92E91E2B92E00E006
:106F800010E0E301C12CD12CE12CF12C9801265FFB
:106F90003C4D2901A8014E505D4D1A01CE010E94C1
:106FA000225DF501EE0DFF1D8083CE0101960E944A
:106FB000325DF201EC0DFD1D60837183828393834A
:106FC000CE0105960E94325DF101EC0DFD1D60833E
:106FD00071838283938329968FEFE81AF80A94E0ED
:106FE000C90ED11C82E0E816F104C1F692E1690EE7
:106FF000711C82E0A80EB11C085F1F4F08311105FB
:1070000009F0BFCFE401CD5BDF4D60E088810E94D5
:107010004A287894DF91CF911F910F91FF90EF90C4
:10702000DF90CF90BF90AF909F908F907F906F90A8
:107030005F904F903F902F90089580E090E00E94E5
:10704000395D21E08D3D9A4B09F020E0822F0895B3
:107050000E941D38882341F083E090E00E94395D52
:1070600080934122909342220895F8946DED7AEB3B
:1070700080E090E00E94695D789408950E94353820
:10708000F894609141227091422283E090E00E9446
:10709000695D78940895CF93DF93EC010E943E5D83
:1070A000CE010196DF91CF910895CF93DF93F894AD
:1070B000C0E0D0E0CE0187709927892B19F480E0D9
:1070C0000E94973660E0CE010E944B382196C11590
:1070D00088E0D80779F760E0809143200E944A2831
:1070E0007894DF91CF9108950C94225DCF93DF9334
:1070F000EC010E94695DCE010296DF91CF91089567
:107100000C94395DCF93DF93EC010E94615DCE0159
:107110000496DF91CF9108950C94325DBC0188E90B
:1071200095E20C947E3EBC0188E995E20C94C93E40
:10713000CF93DF93EB01BC0188E995E20E947E3E8C
:107140004AE050E0BE0188E995E2DF91CF910C94CE
:107150009B3F0F931F93CF93DF931F921F92CDB747
:10716000DEB78B01BC0188E995E249835A830E940E
:107170007E3E49815A81B80188E995E20F900F90CF
:10718000DF91CF911F910F910C949B3F0E949838F3
:1071900088E995E20C94913E0E94A93888E995E22D
:1071A0000C94913ECF92DF92EF92FF92CF93DF93B8
:1071B0001F921F92CDB7DEB76A017B01BC0188E93F
:1071C00095E229833A830E947E3E29813A81B70164
:1071D000A60188E995E20F900F90DF91CF91FF9083
:1071E000EF90DF90CF900C94E9400E94D23888E96C
:1071F00095E20C94913E88E995E20C94913ECF93F0
:10720000DF93C0E7D7E12197CE010E94555900973F
:1072100011F42097C1F70E94ED59CE01DF91CF9173
:1072200008950F931F93CF93DF931F92CDB7DEB7CF
:10723000082F10E0F801E15BFF4D808169830E9417
:10724000C828F801E55BFF4D6981892B39F48081FD
:10725000813061F4662351F010820BC0808181116E
:1072600007C0662329F001E0008302C081E001C06D
:1072700080E00F90DF91CF911F910F91089561E011
:107280000C941139CF93DF93C82FD0E0FE01E15B5E
:10729000FF4D80810E94C828C55BDF4D892B29F4F2
:1072A0008881813039F4188206C08881811102C03A
:1072B00021E0288380E0DF91CF910895CF93DF9381
:1072C000C82FD0E0FE01E15BFF4D80810E94C828FD
:1072D000892B31F4C55BDF4D81E09881913009F451
:1072E00080E0DF91CF910895CF93DF93C82FD0E056
:1072F000FE01E15BFF4D80810E94C828C95BDF4D24
:10730000019731F42881211107C081E0888305C0ED
:107310008881813009F4188280E0DF91CF9108954F
:107320001F93CF93DF93182F0E944327EC01812FE7
:107330000E9443278C0F9D1F95958795DF91CF91D4
:107340001F9108958F929F92AF92BF92CF92DF923A
:10735000EF92FF920F931F93CF93DF93E82EF12CC0
:10736000062F10E0E701CC0FDD1FC00FD11FFE017B
:10737000EE0FFF1FEE0FFF1FE65FFC4D2AE939E914
:1073800049E15FE360817181828193810E943A5675
:107390004B015C010E9453556E01CC0CDD1CF601C3
:1073A000E154FD4D608371836081718180E090E0E4
:1073B0000E9484559B01AC01C501B4010E94EA54AE
:1073C00020E030E040E853E40E943A560E945355D2
:1073D000CD54DD4D6883F601E553FD4D80819181EB
:1073E000880F991FE091D722F091D822E80FF91F5A
:1073F00065917491E701CC0FDD1FC00FD11FCC0F39
:10740000DD1FCC0FDD1FC652DD4D882777FD80952F
:10741000982F0E94865520E030E040E85AE30E9411
:107420003A56688379838A839B83DF91CF911F913A
:107430000F91FF90EF90DF90CF90BF90AF909F9013
:107440008F900895962F20E3829FF0011124E95B2D
:10745000FD4D128E10A211A240E050E060E87FE3E3
:1074600042A353A364A375A316A217A21682178280
:107470001086118610A611A612A613A614A615A68C
:107480009083158616868FEF8287838F0895CF931A
:10749000C82F0E94223A8C2F90E0FC01E659FE4D45
:1074A000A08120E3289FF001299FF00D1124E95BC2
:1074B000FD4DA287B0E0AA0FBB1FAC59BF4D4D9147
:1074C0005C914387548731A130A3FC01EE0FFF1F6D
:1074D000E153FD4D10821182CF910895CF93DF9338
:1074E00090E3899FF0011124E95BFD4D81E08083E9
:1074F000EF01AA96DF019D962081222339F0888131
:107500009981892BC9F73C913111F6CFDF91CF9149
:107510000895CF92DF92EF92FF92CF93DF9390E3A3
:10752000899FE0011124C95BDD4D6A817B818C81DB
:107530009D812E813F81488559850E944F55882322
:1075400069F14A815B816C817D814E835F836887AD
:1075500079876A817B818C819D8126EA3BE944ECB5
:107560005CE30E943A566B017C010E9453556AA766
:107570007BA76AA57BA580E090E00E9484559B01D3
:10758000AC01C701B6010E94EA5420E030E040E8B7
:1075900053E40E943A560E9458556DA7DF91CF914F
:1075A000FF90EF90DF90CF9008951F920F920FB64B
:1075B0000F92112408B60F9218BE09B60F9219BE89
:1075C0000AB60F921ABE0BB60F921BBEEF92FF9235
:1075D0000F931F932F933F934F935F936F937F93DB
:1075E0008F939F93AF93BF93CF93DF93EF93FF93CB
:1075F00042E651E220E030E080E090E07901EE0CDC
:10760000FF1CFA01E80FF91F60816623D1F1E70141
:10761000C80FD91FFE01EE0FFF1FDF01A154BD4DA2
:107620000D911C91E553FD4D60817181600F711FBB
:1076300060837183DE01A754BD4D1C91CD54DD4D97
:107640006881DC9170E06D0F711D6C937C917117F6
:1076500030F4008111810F5F1F4F00831183F70108
:10766000E80FF91FEE0FFF1FE553FD4D608171819B
:107670006835724030F0A081B181A855B240A08336
:10768000B18301968230910509F0BBCF2F5F3F4F48
:107690004E5F5F4F2330310509F0AECFFF91EF9180
:1076A000DF91CF91BF91AF919F918F917F916F911A
:1076B0005F914F913F912F911F910F91FF90EF900C
:1076C0000F900BBE0F900ABE0F9009BE0F9008BE20
:1076D0000F900FBE0F901F901895CF92DF92EF92F0
:1076E000FF922091322330913323E82FF0E0DF0125
:1076F000AA0FBB1FAC5CBC4D0D90BC91A02DAF5729
:10770000BF4FEE0FFF1FEE0FFF1FE65DFC4D69013F
:10771000EE24D7FCE094FE2C0E94C158472F582F2E
:10772000692F772767FD7A95C40ED51EE61EF71ED2
:10773000C082D182E282F382FF90EF90DF90CF90FF
:107740000895FC0124853585F901E058FF4F8081BB
:107750009181329640815181841B950B8F779927B7
:107760000895FC0184859585FC01EE57FF4F20812B
:1077700031813297408151814217530739F0FC0122
:10778000E20FF31F3081832F90E008958FEF9FEF7A
:107790000895FC0184859585FC01EE57FF4F2081FB
:1077A0003181DC01A058BF4F4D915C9142175307C6
:1077B00069F0DC01A20FB31F5C912F5F3F4F2F7761
:1077C000332720833183852F90E008958FEF9FEF3B
:1077D0000895FC0184859585FC01E058FF4FDC018C
:1077E000AE57BF4F2D913C91208331830895DC012A
:1077F0001E96ED91FC911F97818185FFFDCF6083DF
:1078000081E090E00895CF92DF92EF92FF920F9384
:10781000FC01AE2D1282138288EEC82E83E0D82E92
:10782000E12CF12CC482D582E682F78283EC90E2CF
:10783000808391836487758746875787208B318B38
:10784000028BA38B0F91FF90EF90DF90CF90089564
:10785000CF93DF93EC019A01AB01E889F9898A891A
:107860008283E889F9896B896583E889F9897B894D
:107870007183EE85FF851482213482E438078FE01E
:1078800048075105E0F560E070E082E19AE70E9468
:107890007A58345041095109A0E021159EEF39076B
:1078A0009FE14907510540F4A73031F0AF5F220F47
:1078B000331F441F551FF1CFBA01A9019AE07695F5
:1078C0006795579547959A95D1F7EE85FF8546833D
:1078D000EE85FF85A295A07FA195A52BA783EE85B8
:1078E000FF85248128612483EE85FF8533813F7CD9
:1078F000306133830E84DF85C02D43E04D83DF91FB
:10790000CF9108950F931F93CF93DF931F92CDB71D
:10791000DEB78C0129830E94283CD8011E96ED9188
:10792000FC911F97298125830F90DF91CF911F91A3
:107930000F910895DC011E96ED91FC911F97248113
:10794000277E24831E96ED91FC911F9783818F7C67
:10795000806183830895DC011E96ED91FC911F9751
:107960008581662311F0806801C08F778583089533
:1079700081E008951F920F920FB60F92112408B65E
:107980000F9218BE09B60F9219BE0BB60F921BBE0E
:107990002F933F934F935F936F937F938F939F9317
:1079A000AF93BF93EF93FF938091A0096CEA75E2C8
:1079B0000E94F053FF91EF91BF91AF919F918F91F2
:1079C0007F916F915F914F913F912F910F900BBEDF
:1079D0000F9009BE0F9008BE0F900FBE0F901F9022
:1079E00018951F920F920FB60F92112408B60F929E
:1079F00018BE09B60F9219BE0BB60F921BBE2F937D
:107A00003F934F935F936F937F938F939F93AF9326
:107A1000BF93EF93FF938091B00964E175E20E94F8
:107A2000F053FF91EF91BF91AF919F918F917F9113
:107A30006F915F914F913F912F910F900BBE0F90DF
:107A400009BE0F9008BE0F900FBE0F901F901895A3
:107A50001F920F920FB60F92112408B60F9218BE04
:107A600009B60F9219BE0BB60F921BBE2F933F9310
:107A70004F935F936F937F938F939F93AF93BF9336
:107A8000EF93FF938091A0086CE774E20E94F0539B
:107A9000FF91EF91BF91AF919F918F917F916F91E6
:107AA0005F914F913F912F910F900BBE0F9009BEA8
:107AB0000F9008BE0F900FBE0F901F9018951F9249
:107AC0000F920FB60F92112408B60F9218BE09B686
:107AD0000F9219BE0BB60F921BBE2F933F934F937D
:107AE0005F936F937F938F939F93AF93BF93EF9326
:107AF000FF938091B00864EE73E20E94F053FF910F
:107B0000EF91BF91AF919F918F917F916F915F9115
:107B10004F913F912F910F900BBE0F9009BE0F9088
:107B200008BE0F900FBE0F901F9018951F920F92D6
:107B30000FB60F92112408B60F9218BE09B60F9215
:107B400019BE0BB60F921BBE2F933F934F935F93BB
:107B50006F937F938F939F93AF93BF93EF93FF9315
:107B60008091A00A6CE473E20E94F053FF91EF91C0
:107B7000BF91AF919F918F917F916F915F914F9145
:107B80003F912F910F900BBE0F9009BE0F9008BE32
:107B90000F900FBE0F901F901895089508950895A7
:107BA0000895089588E995E20E94A13B892B11F080
:107BB0000E94CD3D80E095E20E94A13B892B11F00F
:107BC0000E94CE3D88E694E20E94A13B892B11F0F1
:107BD0000E94CF3D80ED93E20E94A13B892B11F0E2
:107BE0000E94D03D88E393E20E94A13B892B11F0D3
:107BF0000C94D13D0895CF92DF92EF92FF920F93B4
:107C00001F93CF93DF936C017A01EB01E60EF71E11
:107C100000E010E0CE15DF0561F06991D601ED912D
:107C2000FC910190F081E02DC6011995080F191FF4
:107C3000F1CFC801DF91CF911F910F91FF90EF908D
:107C4000DF90CF900895EF92FF920F931F93CF9301
:107C5000DF938C01FB01C0E0D0E064917F018FEFE6
:107C6000E81AF80A662361F0D801ED91FC910190C1
:107C7000F081E02DC8011995C80FD91FF701EDCF8C
:107C8000CE01DF91CF911F910F91FF90EF9008955A
:107C9000AF92BF92CF92DF92EF92FF920F931F931A
:107CA000CF93DF937C016B01C0E0D0E000E010E0F7
:107CB000D60114968D919C911597C817D90790F409
:107CC000F7010190F081E02DA080B180BE01C601D6
:107CD0000E945B47682FC701F5011995080F191F0E
:107CE0002196E6CFC801DF91CF911F910F91FF90B0
:107CF000EF90DF90CF90BF90AF9008950C94D35445
:107D0000DC01ED91FC910190F081E02D1994DB01F3
:107D1000ED91FC9111970190F081E02DBC01CD0116
:107D200019940F931F93CF93DF93EC016DE00E94A2
:107D3000803E8C016AE0CE010E94803E800F911F40
:107D4000DF91CF911F910F9108950F931F93CF93C0
:107D5000DF93EC010E94233E8C01CE010E94913EF4
:107D6000800F911FDF91CF911F910F9108950F9375
:107D70001F93CF93DF93EC010E94483E8C01CE010C
:107D80000E94913E800F911FDF91CF911F910F9123
:107D900008950F931F93CF93DF93EC010E94D35468
:107DA0008C01CE010E94913E800F911FDF91CF91F7
:107DB0001F910F9108950F931F93CF93DF93EC01C1
:107DC0000E94803E8C01CE010E94913E800F911F47
:107DD000DF91CF911F910F9108950F931F93CF9330
:107DE000DF93EC010E94873E8C01CE010E94913E00
:107DF000800F911FDF91CF911F910F9108958F9266
:107E00009F92AF92BF92CF92DF92EF92FF920F9329
:107E10001F93CF93DF93CDB7DEB7A197CDBFDEBF62
:107E20007C01C42E352FCB01D22E19A221E02D15B5
:107E300010F02AE0D22E8E010F5D1F4F8D2C912C59
:107E4000A12CB12C6C2D732FA50194010E947A589E
:107E50008C2DD29E80191124015011098A3010F402
:107E6000805D01C0895CF8018083211531054105E1
:107E7000510519F0C22ECA01E5CFB801C7010E9411
:107E8000D354A196CDBFDEBFDF91CF911F910F914B
:107E9000FF90EF90DF90CF90BF90AF909F908F902A
:107EA0000895CF92DF92EF92FF920F931F93CF939B
:107EB000DF93EC016A017B012115310579F4E8813A
:107EC000F9810190F081E02D642FDF91CF911F9116
:107ED0000F91FF90EF90DF90CF9019942A303105E9
:107EE000E9F477FF1AC06DE20E94803E8C014427BE
:107EF0005527BA014C195D096E097F092AE0CE01A8
:107F00000E94FF3E800F911FDF91CF911F910F9133
:107F1000FF90EF90DF90CF9008952AE0B701A6017F
:107F2000CE01DF91CF911F910F91FF90EF90DF90E5
:107F3000CF900C94FF3E9A01AB01662757FD6095E8
:107F4000762F0C94513F0F931F93CF93DF93EC0147
:107F50009A01AB01662757FD6095762F0E94513F2D
:107F60008C01CE010E94913E800F911FDF91CF9135
:107F70001F910F9108950F931F93CF93DF93EC01FF
:107F80000E94513F8C01CE010E94913E800F911FB3
:107F9000DF91CF911F910F9108952115310541F483
:107FA000DC01ED91FC910190F081E02D642F19949A
:107FB0000C94FF3E9A01462F50E060E070E00C9474
:107FC000CD3F0F931F93CF93DF93EC019A01462F80
:107FD00050E060E070E00E94CD3F8C01CE010E9435
:107FE000913E800F911FDF91CF911F910F910895C6
:107FF0009A01AB0160E070E00C94CD3F0F931F93AA
:10800000CF93DF93EC019A01AB0160E070E00E9436
:10801000CD3F8C01CE010E94913E800F911FDF91D8
:10802000CF911F910F9108950F931F93CF93DF93DB
:10803000EC010E94CD3F8C01CE010E94913E800F49
:10804000911FDF91CF911F910F9108954F925F92F1
:108050006F927F928F929F92AF92BF92CF92DF9258
:10806000EF92FF920F931F93CF93DF93EC013A01AE
:108070004B01B22E2FEF3FEF4FE75FE4C401B30196
:108080000E9436561816ACF46FEC70E2CE01DF9108
:10809000CF911F910F91FF90EF90DF90CF90BF9005
:1080A000AF909F908F907F906F905F904F900C94C7
:1080B000D3542FEF3FEF4FE75FECC401B3010E94B1
:1080C0004F5587FDE1CF20E030E0A901C401B301A5
:1080D0000E944F5587FF0AC06DE2CE010E94803E8C
:1080E0008C0197FA909497F8909402C000E010E009
:1080F000A12C60E070E080E09FE3AB1441F02DEC38
:108100003CEC4CEC5DE30E943A56A394F6CFA401FC
:1081100093010E94EB546B017C010E9458552B0186
:108120003C010E9484559B01AC01C701B6010E942D
:10813000EA546B017C012AE0B301A201CE010E9446
:10814000FF3E080F191FBB2039F063ED70E2CE012E
:108150000E94D354080F191F7B2C772041F120E097
:1081600030E040E251E4C701B6010E943A566B018B
:108170007C010E9453554B01AA2497FCA094BA2C71
:108180002AE030E0B501A401CE010E94513F080F62
:10819000191FC501B4010E9486559B01AC01C7019E
:1081A000B6010E94EA546B017C017A94D6CFC801D3
:1081B000DF91CF911F910F91FF90EF90DF90CF90C3
:1081C000BF90AF909F908F907F906F905F904F90F7
:1081D00008950C9426400F931F93CF93DF93EC01E7
:1081E0000E9426408C01CE010E94913E800F911F7B
:1081F000DF91CF911F910F910895009729F0BC0155
:1082000080E090E00C94CE5A0895CF93DF9300D095
:108210001F92CDB7DEB79B01AC01611571058105D9
:10822000910569F069833A834B835C830E94CA5A43
:1082300029813A814B815C810E949C5803C060E097
:1082400070E0CB012496CDBFDEBFDF91CF910895C2
:10825000CF92DF92EF92FF926B017C01621773075E
:108260008407950764F4CA01B9016C197D098E0968
:108270009F090E9405416C0D7D1D8E1D9F1DFF9065
:10828000EF90DF90CF9008954F925F926F927F9220
:10829000AF92BF92CF92DF92EF92FF920F931F9314
:1082A000CF93DF93CDB7DEB729013A01621B730B81
:1082B000840B950B2A893B894C895D892A193B09D6
:1082C0004C095D092A8B3B8B4C8B5D8B9B01AC0170
:1082D0006A897B898C899D890E946A58E418F5080F
:1082E00006091709A80197010E949C582A0D3B1DF9
:1082F0004C1D5D1DCA01B901DF91CF911F910F91F6
:10830000FF90EF90DF90CF90BF90AF907F906F90F5
:108310005F904F900895089570E09B01382BC9013C
:108320000895FC01808191810C94ED59CF93DF93E6
:10833000EC0188819981009711F00E94ED59188213
:1083400019821C821D821A821B82DF91CF910895AF
:108350000F931F93CF93DF93EC018B016F5F7F4FE0
:10836000888199810E94D75A009731F08883998338
:108370000A831B8381E001C080E0DF91CF911F91D0
:108380000F910895CF93DF93EC0188819981892B18
:1083900029F02A813B812617370760F4CE010E941D
:1083A000A841882341F0AC81BD81109719F4E88180
:1083B000F981108281E0DF91CF910895EF92FF92D1
:1083C0000F931F93CF93DF93EC017B018A01BA01D6
:1083D0000E94C241811104C0CE010E94964107C093
:1083E0000C831D83B701888199810E94425CCE0174
:1083F000DF91CF911F910F91FF90EF900895FC01B5
:108400001082118212821382148215826115710505
:1084100059F0DB010D900020E9F7AD014150510901
:10842000461B570B0C94DE410895EF92FF920F9379
:108430001F93CF93DF93EC017B018A01BA010E9465
:10844000C241811104C0CE010E94964107C00C8335
:108450001D83B701888199810E94035CCE01DF9161
:10846000CF911F910F91FF90EF900895CF93DF93DD
:10847000EC01FB018617970761F06081718161153E
:10848000710529F0448155810E94DE4102C00E949D
:108490009641CE01DF91CF910895FC0110821182A7
:1084A00012821382148215820C943642CF93DF938A
:1084B000EC016115710561F0FB0101900020E9F705
:1084C000AF0141505109461B570B0E94DE4102C0CB
:1084D0000E949641CE01DF91CF910895CF93DF9313
:1084E0001F921F92CDB7DEB7FC011082118212825B
:1084F00013821482158269831A82BE016F5F7F4FD7
:108500000E9456420F900F90DF91CF9108950F93E4
:108510001F93CF93DF93CDB7DEB72997CDBFDEBFD3
:108520008C01862FF801108211821282138214822C
:10853000158250E0BE016F5F7F4F90E00E94FD5CAE
:10854000BE016F5F7F4FC8010E9456422996CDBF82
:10855000DEBFDF91CF911F910F9108950F931F936D
:10856000CF93DF93CDB7DEB76297CDBFDEBF8C016F
:10857000CB01F801108211821282138214821582BB
:1085800050E0BE016F5F7F4F0E948B5CBE016F5F4A
:108590007F4FC8010E9456426296CDBFDEBFDF9179
:1085A000CF911F910F9108950F931F93CF93DF9356
:1085B000CDB7DEB76197CDBFDEBF8C01CB01F8012F
:1085C00010821182128213821482158250E0BE0141
:1085D0006F5F7F4F0E94FD5CBE016F5F7F4FC801E0
:1085E0000E9456426196CDBFDEBFDF91CF911F91B1
:1085F0000F9108950F931F93CF93DF93CDB7DEB7FD
:10860000A297CDBFDEBF8C01CB01BA01F801108269
:108610001182128213821482158230E0AE014F5F04
:108620005F4F0E94A15CBE016F5F7F4FC8010E9437
:108630005642A296CDBFDEBFDF91CF911F910F9121
:1086400008950F931F93CF93DF93CDB7DEB7A19714
:10865000CDBFDEBF8C01CB01BA01F80110821182BF
:10866000128213821482158230E0AE014F5F5F4F99
:108670000E94D05CBE016F5F7F4FC8010E945642CE
:10868000A196CDBFDEBFDF91CF911F910F910895CD
:10869000EF92FF920F931F93CF93DF93CDB7DEB787
:1086A000A197CDBFDEBF7C01CB01BA01F7011082DB
:1086B0001182128213821482158242E0420F8E01CF
:1086C0000F5F1F4F0E943459BC01C7010E945642E0
:1086D000A196CDBFDEBFDF91CF911F910F91FF908B
:1086E000EF900895EF92FF920F931F93CF93DF9334
:1086F000CDB7DEB7A197CDBFDEBF7C01CB01BA01FC
:10870000F70110821182128213821482158242E0D4
:10871000420F8E010F5F1F4F0E943459BC01C701E9
:108720000E945642A196CDBFDEBFDF91CF911F912F
:108730000F91FF90EF9008950F931F93CF93DF93C6
:108740001F921F92CDB7DEB78C016115710561F0E4
:10875000CB0169837A830E940A5CAC0169817A81CA
:10876000C8010E94154202C00E949641C8010F90A4
:108770000F90DF91CF911F910F910895FC0110820E
:10878000118212821382148215820C949C43EF9200
:10879000FF920F931F93CF93DF93EC017B010C812A
:1087A0001D816115710511F480E016C04115510558
:1087B00091F0040F151FB8010E94C2418823A1F354
:1087C000288139818C819D81B701820F931F0E947E
:1087D000425C0C831D8381E0DF91CF911F910F914B
:1087E000FF90EF900895FB01448155816081718174
:1087F0000C94C7436115710559F0FB0101900020ED
:10880000E9F7AF0141505109461B570B0C94C74380
:1088100080E00895CF93DF931F921F92CDB7DEB70C
:1088200069831A8241E050E0BE016F5F7F4F0E9472
:10883000C7430F900F90DF91CF910895EF92FF9271
:108840000F931F93CF93DF9300D01F92CDB7DEB766
:108850007C01862F4AE050E08E010F5F1F4FB80168
:1088600090E00E948B5CF80101900020E9F7AF01D5
:1088700041505109401B510BB801C7010E94C74329
:108880002496CDBFDEBFDF91CF911F910F91FF9056
:10889000EF900895EF92FF920F931F93CF93DF9382
:1088A000CDB7DEB72897CDBFDEBF7C01CB014AE054
:1088B00050E08E010F5F1F4FB8010E948B5CF801E2
:1088C00001900020E9F7AF0141505109401B510BC5
:1088D000B801C7010E94C7432896CDBFDEBFDF9114
:1088E000CF911F910F91FF90EF900895EF92FF921B
:1088F0000F931F93CF93DF93CDB7DEB72797CDBFED
:10890000DEBF7C01CB014AE050E08E010F5F1F4FBC
:10891000B8010E94FD5CF80101900020E9F7AF0169
:1089200041505109401B510BB801C7010E94C74378
:108930002796CDBFDEBFDF91CF911F910F91FF90A2
:10894000EF900895EF92FF920F931F93CF93DF93D1
:10895000CDB7DEB72E97CDBFDEBF7C01CB01BA010C
:108960002AE030E08E010F5F1F4FA8010E94A15C3A
:10897000F80101900020E9F7AF0141505109401B77
:10898000510BB801C7010E94C7432E96CDBFDEBF71
:10899000DF91CF911F910F91FF90EF900895EF928B
:1089A000FF920F931F93CF93DF93CDB7DEB72D9731
:1089B000CDBFDEBF7C01CB01BA012AE030E08E01E1
:1089C0000F5F1F4FA8010E94D05CF80101900020AA
:1089D000E9F7AF0141505109401B510BB801C701E4
:1089E0000E94C7432D96CDBFDEBFDF91CF911F916F
:1089F0000F91FF90EF900895EF92FF920F931F93C6
:108A0000CF93DF93CDB7DEB76497CDBFDEBF7C01D8
:108A1000CB01BA018E010F5F1F4F22E044E00E949C
:108A20003459FC0101900020E9F7AF014150510990
:108A3000481B590BBC01C7010E94C7436496CDBFB8
:108A4000DEBFDF91CF911F910F91FF90EF900895BE
:108A5000EF92FF920F931F93CF93DF93CDB7DEB7C3
:108A60006497CDBFDEBF7C01CB01BA018E010F5FE1
:108A70001F4F22E044E00E943459FC010190002085
:108A8000E9F7AF0141505109481B590BBC01C7011F
:108A90000E94C7436496CDBFDEBFDF91CF911F9187
:108AA0000F91FF90EF900895EF92FF920F931F9315
:108AB000CF93DF93EC017B016115710511F480E028
:108AC0001BC0CB010E940A5C0097A9F00C811D819C
:108AD000080F191FB801CE010E94C241882379F303
:108AE000288139818C819D81B701820F931F0E945B
:108AF000035C0C831D8381E0DF91CF911F910F9167
:108B0000FF90EF900895CF93DF93EC01FB01448138
:108B10005581608171810E94C743811103C0CE01DC
:108B20000E949641CE01DF91CF910895CF93DF93BC
:108B3000EC016115710569F0FB0101900020E9F776
:108B4000AF0141505109461B570B0E94C743811189
:108B500003C0CE010E949641CE01DF91CF910895CE
:108B6000CF93DF93EC010E940A44811103C0CE0130
:108B70000E949641CE01DF91CF910895CF93DF936C
:108B8000EC010E941E44811103C0CE010E94964157
:108B9000CE01DF91CF910895CF93DF93EC010E9436
:108BA0004A44811103C0CE010E949641CE01DF915B
:108BB000CF910895CF93DF93EC010E947644811109
:108BC00003C0CE010E949641CE01DF91CF9108955E
:108BD000CF93DF93EC010E94A244811103C0CE0128
:108BE0000E949641CE01DF91CF910895CF93DF93FC
:108BF000EC010E94CF44811103C0CE010E94964136
:108C0000CE01DF91CF910895CF93DF93EC010E94C5
:108C1000FC44811103C0CE010E949641CE01DF9138
:108C2000CF910895CF93DF93EC010E9428458111E5
:108C300003C0CE010E949641CE01DF91CF910895ED
:108C4000CF93DF93EC010E945445811103C0CE0104
:108C50000E949641CE01DF91CF910895CF93DF938B
:108C6000DC01ED91FC91EB01A881B981309711F005
:108C70001097C9F4109759F0EB012C813D81232BFB
:108C800031F08C9190E091958195910914C03097C5
:108C900081F0DC0114968D919C911597892B49F0F8
:108CA000808190E008C0BD01CF01DF91CF910C948D
:108CB000395C80E090E0DF91CF910895FC01448120
:108CC0005581FB01248135814217530741F40E94ED
:108CD0002E4631E0892B09F030E0832F089580E0A3
:108CE0000895FC0124813581232B31F431E0611595
:108CF0007105A1F0FB0108C0FC0180819181611523
:108D0000710531F431E0FC018081882339F005C020
:108D10000E94395C31E0892B09F030E0832F0895FF
:108D20000E942E46892F881F8827881F08950E9439
:108D30002E4621E0181619060CF020E0822F089527
:108D40000E942E4621E0181619060CF420E0822F0E
:108D500008950E942E46892F8095881F8827881F96
:108D60000895EF92FF920F931F93CF93DF9386178F
:108D7000970719F1FC0124813581EB014C815D815C
:108D800024173507E1F4232BC1F0FC010081118188
:108D9000EB010990D881C02DF80181918F018823C2
:108DA00061F090E00E94F35B7C01899190E00E9469
:108DB000F35BE816F90681F302C081E001C080E0B0
:108DC000DF91CF911F910F91FF90EF900895FA01DD
:108DD000DB0114964D915C911597DC0114962D9151
:108DE0003C911597241B350B2E173F0788F08D916A
:108DF0009C91009769F0DB016D917C916115710583
:108E000039F08E0F9F1F0E94495C31E0892B09F0D9
:108E100030E0832F0895FC0144815581FB012481BA
:108E200035814217530720F040E050E00C94E746AC
:108E300080E00895FC0184819581DB0114964D91B9
:108E40005C9115978417950798F020813181211541
:108E5000310571F06D917C916115710549F0841BAC
:108E6000950B820F931F0E94395C31E0892B09F02A
:108E700030E0832F0895DC0114962D913C911597D5
:108E80006217730728F4ED91FC91E60FF71F4083FA
:108E90000895FC01848195816817790720F4808109
:108EA0009181009729F41092302680E396E208958C
:108EB000860F971F0895FC0124813581621773077F
:108EC00048F480819181009729F0FC01E60FF71F9B
:108ED0008081089580E008950C945B470F931F9361
:108EE000CF93DF93EB0141155105E9F02097D9F0BD
:108EF000FC016481758126173707A0F4621B730B90
:108F00008A01015011096017710708F48B01FC01F7
:108F100060817181620F731FA801CE010E94575CAE
:108F2000C00FD11F1882DF91CF911F910F9108952B
:108F3000CF93DF93FC01848195814817590768F42A
:108F4000C081D18170E0CE01840F951F0E942E5CFC
:108F5000009719F08C1B9D0B02C08FEF9FEFDF91E4
:108F6000CF91089540E050E00C949847CF93DF9361
:108F7000FC01848195814817590778F4C081D1811B
:108F8000FB0160817181CE01840F951F0E94715C8D
:108F9000009719F08C1B9D0B02C08FEF9FEFDF91A4
:108FA000CF91089540E050E00C94B647DF92EF92E5
:108FB000FF920F931F93CF93DF93EC018C819D81E0
:108FC0004817590718F08FEF9FEF19C08A010F5FFC
:108FD0001F4FE881F981E00FF11FD0801082E880F7
:108FE000F98070E0C7010E94665CF701E00FF11F95
:108FF000D082009741F328813981821B930BDF9146
:10900000CF911F910F91FF90EF90DF900895FC0199
:1090100044815581415051090C94D647AF92BF927B
:10902000CF92DF92EF92FF920F931F93CF93DF9334
:109030007B01EA01FB01448155814115510569F12C
:10904000FC01248135812115310539F124173507BB
:1090500020F1C217D30710F0E9012197FC0100812C
:109060001181C801AA24AA94BB24BA946801CC0E29
:10907000DD1EC816D906A0F0F701608171810E943B
:10908000715C009769F0BC01601B710BC617D707B4
:1090900008F4B50101965B01ECCF8FEF9FEF01C0A3
:1090A000C501DF91CF911F910F91FF90EF90DF905D
:1090B000CF90BF90AF900895FC0144815581FB0192
:1090C00024813581421B530B0C940E48BF92CF92E2
:1090D000DF92EF92FF920F931F93CF93DF936C0178
:1090E0007B01EA0189012417350720F48D2FE9015E
:1090F000042F182F60EA70E2C6010E94FF41D701D9
:1091000014962D913C9115972C173D07C8F0201708
:10911000310708F48901D701ED91FC911197E00F17
:10912000F11FB08010826D917C916C0F7D1FC60184
:109130000E945642E701E881F981E00FF11FB082F9
:10914000C601DF91CF911F910F91FF90EF90DF90BB
:10915000CF90BF900895DC01ED91FC91309729F4F8
:109160000895861301C04083319680818111F9CF23
:1091700008952F923F924F925F926F927F928F92BB
:109180009F92AF92BF92CF92DF92EF92FF920F9396
:109190001F93CF93DF93EC015B017A014C805D80DC
:1091A0004114510409F4C5C0FB0164807580611449
:1091B000710409F4BEC0FA01C480D580C618D7086E
:1091C00008811981C114D104C1F4E5016881798154
:1091D000C8010E94715CEC01009709F4AAC0F70174
:1091E0006081718144815581CE010E94135CF70139
:1091F000048115810C0F1D1FE8CFD7FC05C0FB01B2
:1092000020803180420143C03801F50160817181C5
:10921000C8010E94715C1C01009719F12101401ADC
:10922000510AA201B801C3010E94135C460C571CED
:10923000F7016081718144815581C2010E94135CF4
:10924000F70164807580640C751CF501048115813B
:10925000020D131D4C815D814C0D5D1D4C835D83A2
:10926000D4CFB801C301DF91CF911F910F91FF902F
:10927000EF90DF90CF90BF90AF909F908F907F90B6
:109280006F905F904F903F902F900C94425CB10193
:10929000C8010E94715C009731F08C01060D171D0A
:1092A0008C0C9D1CF4CF8414950409F442C08A816F
:1092B0009B818815990530F4B401CE010E94A84124
:1092C0008823B9F14C815D814150510957FD31C06E
:1092D000B501CE010E940E488C0197FD2AC08881FD
:1092E0009981F50124813581200F311F820F931F51
:1092F0004C815D81421B530BBC018C0D9D1D0E9456
:109300001C5C2C803D802C0C3D1C2C823D82E88115
:10931000F981E20DF31D108288819981F701608146
:10932000718144815581800F911F0E94135CA801B7
:10933000CBCFDF91CF911F910F91FF90EF90DF90F6
:10934000CF90BF90AF909F908F907F906F905F90E5
:109350004F903F902F900895CF93DF93EC019B01A6
:10936000BA014C815D812417350718F56115710527
:1093700001F1C901860F971F4817590718F4BA0160
:10938000621B730B88819981461B570B4C835D834D
:10939000421B530B620F731F680F791F820F931FBD
:1093A0000E94575CE881F9814C815D81E40FF51FD3
:1093B0001082DF91CF910895FC014481558164179B
:1093C000750720F4461B570B0C94AC490895CF93B6
:1093D000DF93FC01C081D181209741F088818823EF
:1093E00029F090E00E94F35B8993F8CFDF91CF9151
:1093F0000895CF93DF93FC01C081D181209741F084
:109400008881882329F090E00E94FB5B8993F8CF44
:10941000DF91CF910895AF92BF92CF92DF92EF92FA
:10942000FF920F931F93CF93DF937C01DC01CD90CC
:10943000DC901197C114D104E1F11496CD91DC9127
:1094400015972097B1F156018501BFEFAB1ABB0A02
:10945000F801808190E00E94EB5B892BA9F72197AE
:10946000CC0DDD1DB8808B2D90E00E94EB5B892B2D
:1094700081F4AE014F5F5F4F401B510BE7014C83FE
:109480005D83C016D10650F4B801C6010E94135C7A
:1094900005C0C017D10768F32197E4CFD701ED913C
:1094A000FC9111971496CD90DC901597EC0DFD1D55
:1094B0001082DF91CF911F910F91FF90EF90DF907D
:1094C000CF90BF90AF900895FC018081918100976B
:1094D00011F00C94C45B60E070E0CB010895FC01D6
:1094E00080819181009711F00C94C05B60E070E086
:1094F000CB0108951F920F920FB60F92112408B658
:109500000F9218BE09B60F9219BE0AB60F921ABE74
:109510000BB60F921BBE2F923F924F925F926F92AB
:109520007F928F929F92AF92BF92CF92DF92EF92F3
:10953000FF920F931F932F933F934F935F936F93DC
:109540007F938F939F93AF93BF93EF93FF93CF93AB
:10955000DF9300D01F92CDB7DEB78091532090915A
:10956000542080933803909339030FEF17E0009352
:1095700053201093542027E432E22B833C8334E3BE
:10958000A32E33E2B32E46E2C42E43E2D42E5AE297
:10959000852E53E2952E62E2E62E63E2F62E00E07F
:1095A00010E0612C712CAB81BC812C90222009F43D
:1095B000AAC09A964D905C909B9798964D915C911D
:1095C0009997440D551D98964D935C9399979C9649
:1095D0003C909C979D968C919D979C963C919C97D6
:1095E00090E0830F911D9C968C939C979C965C9029
:1095F0009C97531448F49896ED91FC919997319665
:109600009896ED93FC939997EB81FC8160A571A5E9
:109610006835F2E07F0708F4CCC0AB81BC815C9177
:10962000513009F4EEC098968D919C919997885588
:10963000924098968D939C939997F801E95BFD4D24
:1096400081A180A3BAC0120135942794F201F59547
:10965000E795F595E795F595E795F595E795F595F2
:10966000E79521014E1A5F0AF595E7954E1A5F0AB4
:10967000D501ED91FC91EF3FF10509F442C0D6010F
:109680002D903C90D7014D915C9149835A834218AB
:109690005308B101641B750BD4012D913D914D917F
:1096A0005C91DB010E94EA58BB2797FDBA95A92F70
:1096B000982F872F480E591E9F01D2010E94C15832
:1096C000BB2797FDBA95A92F982F872F2101480E08
:1096D000591ED6014D925C9289819A81481A590A85
:1096E0009F01D2010E94C158BB2797FDBA95A92FAF
:1096F000982F872F49805A80480E591EF7014082C3
:109700005182640C751CAB81BC81D096AB83BC8349
:10971000005D1F4FF2E0AF0EB11C22E0C20ED11C63
:1097200034E0830E911C82E0E80EF11C0036110536
:1097300009F039CF91E0691A98EF790A77FC64C093
:109740006114A0E17A060CF457C00FEF1FE00093FC
:109750005320109354202496CDBFDEBFDF91CF91CC
:10976000FF91EF91BF91AF919F918F917F916F91F9
:109770005F914F913F912F911F910F91FF90EF902B
:10978000DF90CF90BF90AF909F908F907F906F9021
:109790005F904F903F902F900F900BBE0F900ABE9E
:1097A0000F9009BE0F9008BE0F900FBE0F901F9034
:1097B0001895F801E95BFD4D80A1AB81BC819896BD
:1097C0002D913C919997220F331F1B96ED91FC919F
:1097D0001C97E20FF31F459054905594479490E0E6
:1097E00001978034910518F0412C512C41CFFC0198
:1097F000E250FF4F0C94BB5860925320709254205B
:10980000AACFFD0110827FCF1092532010925420D6
:10981000A2CFF201F595E795559447945594479456
:109820005594479455944794559447949F0124190F
:10983000350929011DCF120135942794042C452C9C
:10984000000C441C5508000C441C551CD101A419E3
:10985000B5092D010DCF559447940ACFC2019595B6
:109860008795042C452C000C441C5508000C441C06
:10987000551C480E591EFCCEA2015595479555948E
:1098800047945594479455944794559447945594C8
:109890004794440E551EECCEF201F595E795B201C2
:1098A00075956795759567957595679575956795A0
:1098B000759567952F01460E571E75956795460E4F
:1098C000571ED6CE1201359427945594479455943B
:1098D00047945594479455944794420C531CC8CED2
:1098E000D201B595A7959201359527953595279580
:1098F00035952795359527952D01420E531E3595A3
:10990000279535952795420E531EB2CEB201759517
:109910006795C201959587959595879595958795B6
:10992000959587952B01480E591E95958795480E5C
:10993000591E9ECE120135942794A2015595479544
:109940005595479555954795559547952101440E51
:10995000551EFA01F595E7954E0E5F1E55954795F4
:1099600055954795440E551E83CE92013595279502
:1099700029015594479455944794420E531E78CE2E
:10998000B20175956795DB01B595A795B595A79536
:10999000A60FB71F042C452C000C441C5508000CC6
:1099A000441C551C4A0E5B1E63CE5594479412010D
:1099B0003594279435942794420C531C359427945E
:1099C00035942794420C531C53CEA20155954795CC
:1099D000CA019595879595958795480F591F959537
:1099E000879595958795480F591F042C452C000C99
:1099F000441C5508000C441C551C440E551E38CE02
:109A000055944794C2019595879595958795480EED
:109A1000591E95958795480E591E2ACEF201F59547
:109A2000E795F595E7951201359427943594279499
:109A30003594279435942794359427944E1A5F0AC9
:109A400042185308359427944218530811CEB20196
:109A50007595679575956795C201861B970B55940B
:109A600047945594479455944794559447945594E6
:109A700047949C01241935092901FACD92013595A5
:109A8000279535952795F201E21BF30B042C452C05
:109A9000000C441C5508000C441C551CAF01441913
:109AA00055092A01E5CDD201B595A795B595A7959C
:109AB0004A1A5B0ADDCDA201559547955595479504
:109AC000B201641B750B042C452C000C441C55087A
:109AD000000C441C551C460E571ECACD92013595EC
:109AE000279535952795F201E21BF30B5594479482
:109AF0005594479455944794559447945594479456
:109B00004E0E5F1EB5CDB20175956795759567953B
:109B100075956795C201861B970B75956795861B92
:109B2000970B042C452C000C441C5508000C441CBD
:109B3000551CDC01A419B5092D019ACDA20155953A
:109B400047955595479555954795441A550A559506
:109B50004795441A550A8CCD920135952795359530
:109B60002795359527951901359427943594279491
:109B7000421A530A4218530835942794421853083E
:109B800077CDF201F595E795F595E795F595E7958C
:109B90004E1A5F0AF595E795F595E7954E1A5F0A17
:109BA00067CDA2015595479555954795559547958C
:109BB000B201641B750B042C452C000C441C550889
:109BC000000C441C551CDB01A419B5092D0150CD16
:109BD000120135942794359427943594279442188C
:109BE000530846CDF201F595E795F595E795F5957E
:109BF000E795F595E7954E1A5F0A9F0135952795EC
:109C000035952795421A530AF595E7954E1A5F0A3E
:109C10002FCDD201B595A795B595A795B595A795E3
:109C2000B595A7954A1A5B0AB595A7954A1A5B0A96
:109C30001FCDC201959587959595879595958795A3
:109C400095958795481A590A95958795959587957D
:109C5000481A590A0DCDB2017595679575956795A6
:109C60007595679575956795461A570A01CDA201B6
:109C700055954795559547955595479555954795CC
:109C800055954795441A550A55954795441A550ACE
:109C9000EFCC12013594279435942794559447942A
:109CA00055944794559447945594479455944794A4
:109CB000B101641975092B01DBCC9201359527950B
:109CC00035952795042C452C000C441C5508000C98
:109CD000441C551CD901A419B5092D01C9CC5594B2
:109CE000479455944794C4CCC20195958795959512
:109CF0008795042C452C000C441C5508000C441C72
:109D0000551C480E591EB4CCF201F595E795F59512
:109D1000E795559447945594479455944794559492
:109D20004794559447944E0E5F1EA2CC5594479489
:109D300055944794A2015595479555954795440EDE
:109D4000551E5595479555954795441A550A90CCFB
:109D5000B20175956795759567952B015594479454
:109D600055944794460E571E83CC5594479455946A
:109D700047941DCE55944794920135952795359576
:109D80002795421A530A3595279535952795421AF6
:109D9000530A6ECCF201F595E795CF01959587951D
:109DA00095958795E81BF90B042C452C000C441C59
:109DB0005508000C441C551CDF01A419B5092D01E0
:109DC00057CC55944794A20155954795559547957D
:109DD000441A550A4DCC120135942794B10175955A
:109DE000679575956795261A370A042C452C000C43
:109DF000441C5508000C441C551C420C531C38CC08
:109E0000D201B595A795920135952795359527955A
:109E100035952795359527952D01421A530A359585
:109E20002795421A530A24CCF201F595E795C20111
:109E3000959587959595879595958795959587950A
:109E40002F01481A590A9595879595958795481A2F
:109E5000590A0ECCB201759567955594479455945F
:109E600047945594479455944794AB014419550928
:109E70002A01FECB559447945594479455944794A2
:109E8000F201F595E795F595E7954E1A5F0AF0CB47
:109E9000D201B595A795B595A795B595A795042C2D
:109EA000452C000C441C5508000C441C551CBD01DD
:109EB000641975092B01DCCB55944794559447944C
:109EC00055944794D5CB1201359427943594279413
:109ED00035942794042C452C000C441C5508000C88
:109EE000441C551C420C531CC3CB9201359527953D
:109EF000359527953595279529015594479455947F
:109F00004794420E531EB4CB5594479455944794AE
:109F10005594479477CD5594479455944794A2010E
:109F20005595479555954795441A550AA1CB120169
:109F3000359427943594279489CB55944794559418
:109F4000479455944794559447945594479490CB8F
:109F500055944794559447945594479455944794F1
:109F6000C2019595879595958795481A590A80CB92
:109F700055944794559447945594479455944794D1
:109F800077CBA2015595479555954795559547959A
:109F9000559547952A015594479455944794440EF6
:109FA000551E66CB9201022E232F000C221F330B6D
:109FB000000C221F331F421A530A5ACB042C452C83
:109FC000000C441C5508000C441C551C51CB1201BC
:109FD0003594279435942794359427943594279471
:109FE000359427944218530843CB9C01462F50E0E8
:109FF000415051094034510518F080E090E0089537
:10A00000FA01E25CFE4F0C94BB58959587959595A7
:10A010008795959587959595879595958795B90198
:10A02000681B790BCB010895AC0155954795559563
:10A030004795559547955595479555954795841B53
:10A04000950B55954795841B950B0895FC01F59547
:10A05000E795F595E795F595E795F595E795DC0195
:10A06000AE1BBF0BCD010895BC0175956795759525
:10A0700067957595679575956795C901861B970BCB
:10A080007595679575956795861B970B0895AC0137
:10A0900055954795559547955595479555954795A8
:10A0A000841B950B55954795841B950B0895BC0112
:10A0B0007595679575956795759567957595679588
:10A0C000861B970B9B013595279535952795821B08
:10A0D000930B75956795861B970B089595958795B6
:10A0E0009595879595958795F901E81BF90BCF0113
:10A0F0000895DC01B595A795B595A795B595A79554
:10A10000AC014A1B5B0BCA01022E232F000C221F3D
:10A11000330B000C221F331F821B930B0895FC018D
:10A12000F595E795F595E795F595E7958E1B9F0BCA
:10A13000F595E795F595E7958E1B9F0B08959595F9
:10A1400087959595879595958795AC0155954795F4
:10A1500055954795D901A81BB90BCD01841B950BCB
:10A1600055954795841B950B0895BC01759567958A
:10A170007595679575956795861B970B759567958A
:10A18000861B970B0895DC01B595A795B595A79506
:10A19000B595A7958A1B9B0BB595A7958A1B9B0B1D
:10A1A000022E232F000C221F330B000C221F331F03
:10A1B000821B930B08959595879595958795F90141
:10A1C000E81BF90BCF0135952795359527953595E2
:10A1D00027953595279535952795820F931F0895D7
:10A1E000AC015595479555954795BC01641B750B7A
:10A1F000CB01022E232F000C221F330B000C221F39
:10A20000331F820F931F0895DC01B595A795B5956F
:10A21000A7959C012A1B3B0BC9010895959587952D
:10A2200095958795F901E81BF90BCF01022E232F95
:10A23000000C221F330B000C221F331F821B930BB9
:10A240000895BC017595679575956795AC01461B9A
:10A25000570BCA013595279535952795359527953F
:10A260003595279535952795821B930B08959595E0
:10A27000879595958795A901559547955595479546
:10A2800055954795559547955595479563CF959520
:10A290008795AC015595479555954795840F951F22
:10A2A00055954795840F951F089595958795FC01C1
:10A2B000F595E795F595E7958E0F9F1FF595E79531
:10A2C000F595E7958E0F9F1F022E232F000C221F5E
:10A2D000330B000C221F331F820F931F0895959597
:10A2E0008795AC015595479555954795840F951FD2
:10A2F0005595479555954795840F951F0895AC0141
:10A3000055954795CA019595879595958795840F9D
:10A31000951F022E232F000C221F330B000C221F2F
:10A32000331F820F931F089535952795C901959581
:10A33000879595958795820F931F08959595879595
:10A3400035952795359527953595279535952795F5
:10A35000820F931FD901B595A7958A0F9B1F35953D
:10A36000279535952795820F931F08959595879585
:10A3700035952795359527953595279535952795C5
:10A38000820F931F35952795820F931F08959595FA
:10A390008795359527953595279535952795359545
:10A3A0002795820F931F3595279535952795820F11
:10A3B000931F0895FC01F595E795959587959595DB
:10A3C000879595958795959587958E0F9F1F0895ED
:10A3D00095958795359527953595279535952795A5
:10A3E0003595279535952795820F931F3595279598
:10A3F000820F931F0895BC01759567959595879574
:10A400009595879595958795959587959595879534
:10A41000860F971F0895AC0155954795082E892FF3
:10A42000000C881F990B000C881F991F840F951F23
:10A43000089595958795089595958795022E232FD4
:10A44000000C221F330B000C221F331F821B930BA7
:10A450000895959587953595279535952795359543
:10A4600027953595279535952795821B930B08954C
:10A470009595879535952795359527953595279504
:10A480003595279535952795821B930B35952795FF
:10A49000821B930B0895959587953595279535954E
:10A4A00027953595279535952795821B930B08950C
:10A4B00095958795359527953595279535952795C4
:10A4C00035952795821B930B3595279535952795BF
:10A4D000821B930B0895959587953595279535950E
:10A4E00027953595279535952795821B930B35959F
:10A4F0002795821B930B089595958795DC01B5955B
:10A50000A795B595A7958A1B9B0B022E232F000CB0
:10A51000221F330B000C221F331F820F931F08953D
:10A52000959587959C013595279535952795821B9F
:10A53000930B089595958795FC01F595E795F5950D
:10A54000E7958E1B9F0B022E232F000C221F330B2F
:10A55000000C221F331F821B930B0895959587953E
:10A56000BC017595679575956795861B970B7595D5
:10A57000679575956795861B970B089595958795B3
:10A5800095958795AECE3595279535952795C90133
:10A590009595879595958795820F931F0895959525
:10A5A000879595958795DC01B595A795B595A79560
:10A5B0008A0F9B1FB595A795B595A7958A1B9B0BF1
:10A5C0000895BC01759567957595679595958795DF
:10A5D0009595879595958795959587959595879563
:10A5E000860F971F0895FC01F595E795F595E7957A
:10A5F000082E892F000C881F990B000C881F991FAB
:10A600008E0F9F1F08959595879595958795089529
:10A610009595879595958795022E232F000C221FDF
:10A62000330B000C221F331F821B930B089595954B
:10A6300087959595879535952795359527953595E2
:10A6400027953595279535952795821B930B08956A
:10A650009595879595958795359527953595279562
:10A66000359527953595279535952795821B930B1D
:10A6700035952795821B930B08959595879595950C
:10A6800087959C013595279535952795821B930BCA
:10A690000895959587959595879595958795F9CD85
:10A6A000359527953595279535952795C901959524
:10A6B000879595958795820F931F0895DC01B59531
:10A6C000A795B595A795B595A795082E892F000C48
:10A6D000881F990B000C881F991F8A0F9B1F0895D4
:10A6E00095958795959587959595879508959595D1
:10A6F00087959595879595958795022E232F000C24
:10A70000221F330B000C221F331F821B930B089553
:10A71000959587959595879595958795FC01F595E0
:10A72000E795F595E7958E1B9F0B08953595279531
:10A73000359527953595279535952795C901959593
:10A74000879595958795820F931F08959595879581
:10A750009595879595958795959587950895959560
:10A760008795959587959595879595958795BC013E
:10A770007595679575956795861B970B08959595C3
:10A7800087959595879595958795959587959595B1
:10A7900087950895082E892F000C881F990B000CAF
:10A7A000881F991F0895082E892F000C881F990B68
:10A7B000000C881F991F281B390BC90108950895A3
:10A7C0000E9496260E94872B0E948C2CFDCF8091A0
:10A7D0005A2090915B208093D7229093D82208959D
:10A7E000FB01E058FF4F408151819A012F5F3F4F9D
:10A7F0002F773327DB01AE57BF4F0D90BC91A02DB3
:10A800002A173B0731F0DB01A40FB51F8C9320837F
:10A8100031830895CF93DF9310929A2510929B2550
:10A8200088EE93E0A0E0B0E080939C2590939D2576
:10A83000A0939E25B0939F2523EC30E2209398258A
:10A84000309399254CEA55E24093A4255093A525D1
:10A8500060EA79E06093A6257093A725C0E6D6E06C
:10A86000C093A825D093A925F4E0F093AA25E8E0A9
:10A87000E093AB25109202251092032580930425C6
:10A8800090930525A0930625B093072520930025D6
:10A890003093012544E155E240930C2550930D255A
:10A8A00060EB79E060930E2570930F25C09310251F
:10A8B000D0931125D0E4D0931225C0E8C09313257E
:10A8C00010926A2410926B2480936C2490936D24D0
:10A8D000A0936E24B0936F2420936824309369244E
:10A8E0004CE754E2409374245093752460EA78E076
:10A8F000609376247093772440E456E04093782464
:10A9000050937924F0937A24E0937B241092D223FD
:10A910001092D3238093D4239093D523A093D6234E
:10A92000B093D7232093D0233093D12364EE73E2E6
:10A930006093DC237093DD2360EB78E06093DE238B
:10A940007093DF234093E0235093E123D093E223DD
:10A95000C093E32310923A2310923B2380933C232D
:10A9600090933D23A0933E23B0933F23209338231D
:10A9700030933923ACE4B3E2A0934423B09345234E
:10A9800080EA9AE0809346239093472320E836E0BC
:10A990002093482330934923F0934A23E0934B2399
:10A9A000DF91CF9108956115710589F0DB010D905C
:10A9B0000020E9F7AD0141505109461B570BFC013E
:10A9C0000190F081E02D0280F381E02D199480E068
:10A9D00090E008955058BB27AA270ED00DC1FED095
:10A9E00030F003D120F031F49F3F11F41EF4F3C096
:10A9F0000EF4E095E7FBE9C0E92F0FD180F3BA1719
:10AA0000620773078407950718F071F49EF527C154
:10AA10000EF4E0950B2EBA2FA02D0B01B901900179
:10AA20000C01CA01A0011124FF27591B99F0593FBD
:10AA300050F4503E68F11A16F040A22F232F342F05
:10AA40004427585FF3CF469537952795A795F04053
:10AA50005395C9F77EF41F16BA0B620B730B840B68
:10AA6000BAF09150A1F0FF0FBB1F661F771F881F20
:10AA7000C2F70EC0BA0F621F731F841F48F4879578
:10AA800077956795B795F7959E3F08F0B3CF939567
:10AA9000880F08F09927EE0F97958795089571D044
:10AAA00008F481E0089504D06894B111D9C00895E4
:10AAB000BCD088F09F5790F0B92F9927B751A0F0DC
:10AAC000D1F0660F771F881F991F1AF0BA95C9F742
:10AAD00012C0B13081F0C3D0B1E00895C0C0672F7B
:10AAE000782F8827B85F39F0B93FCCF386957795F2
:10AAF0006795B395D9F73EF49095809570956195DB
:10AB00007F4F8F4F9F4F0895E89409C097FB3EF405
:10AB100090958095709561957F4F8F4F9F4F9923AA
:10AB2000A9F0F92F96E9BB279395F6958795779528
:10AB30006795B795F111F8CFFAF4BB0F11F460FFE8
:10AB40001BC06F5F7F4F8F4F9F4F16C0882311F040
:10AB500096E911C0772321F09EE8872F762F05C054
:10AB6000662371F096E8862F70E060E02AF09A95EF
:10AB7000660F771F881FDAF7880F9695879597F9E4
:10AB80000895990F0008550FAA0BE0E8FEEF16167E
:10AB90001706E807F907C0F012161306E407F507D1
:10ABA00098F0621B730B840B950B39F40A2661F045
:10ABB000232B242B252B21F408950A2609F4A140E8
:10ABC000A6958FEF811D811D089597F99F6780E8F5
:10ABD00070E060E008959FEF80EC089500240A94EF
:10ABE0001616170618060906089500240A94121668
:10ABF0001306140605060895092E0394000C11F49B
:10AC0000882352F0BB0F40F4BF2B11F460FF04C047
:10AC10006F5F7F4F8F4F9F4F089557FD9058440FA0
:10AC2000551F59F05F3F71F04795880F97FB991FAB
:10AC300061F09F3F79F08795089512161306140668
:10AC4000551FF2CF4695F1DF08C0161617061806F5
:10AC5000991FF1CF86957105610508940895E894D0
:10AC6000BB2766277727CB0197F908958ADF08F479
:10AC70008FEF08950BD0C0CFB1DF28F0B6DF18F00A
:10AC8000952309F0A2CFA7CF1124EACFC6DFA0F306
:10AC9000959FD1F3950F50E0551F629FF001729F71
:10ACA000BB27F00DB11D639FAA27F00DB11DAA1F90
:10ACB000649F6627B00DA11D661F829F2227B00DDD
:10ACC000A11D621F739FB00DA11D621F839FA00D68
:10ACD000611D221F749F3327A00D611D231F849FB8
:10ACE000600D211D822F762F6A2F11249F5750400F
:10ACF0008AF0E1F088234AF0EE0FFF1FBB1F661FAA
:10AD0000771F881F91505040A9F79E3F510570F062
:10AD10005CCFA6CF5F3FECF3983EDCF3869577954A
:10AD20006795B795F795E7959F5FC1F7FE2B880F5D
:10AD3000911D9695879597F90895FA01EE0FFF1FDB
:10AD400030962105310599F16115710561F480385E
:10AD5000BFE39B0749F168949038810561F0803822
:10AD6000BFEF9B0741F0992342F5FF3FE105310515
:10AD7000210511F1E8940894E795D901AA2329F453
:10AD8000AB2FBE2FF85FD0F310C0FF5F70F4A69515
:10AD9000E0F7F73950F019F0FF3A38F49F779F93B6
:10ADA0000CD00F9007FC905808953EF014CF60E04F
:10ADB00070E080E89FE308954FE79F775F934F939C
:10ADC0003F932F939ED02F913F914F915F9152DFF0
:10ADD00005C019F40EF0F9CE42CFFDCE26DFC8F340
:10ADE0009638C0F707F80F92E8942BE33AEA48EB5D
:10ADF0005FE74EDF0F920F920F924DB75EB70F9243
:10AE0000C0D0ECEFF2E016D04F915F91EF91FF913F
:10AE1000E595EE1FFF1F49F0FE57E0684427EE0F4F
:10AE2000441FFA95E1F74195550B32D00F9007FE7C
:10AE300026C00895DF93CF931F930F93FF92EF9255
:10AE4000DF927B018C01689405C0DA2EEF011EDFD2
:10AE5000FE01E894A5912591359145915591AEF368
:10AE6000EF01CADDFE019701A801DA9479F7DF90BE
:10AE7000EF90FF900F911F91CF91DF9108959B016B
:10AE8000AC0160E070E080E89FE3AEC09ECE14C1EC
:10AE9000CCDEE8F39923D9F3940F511DBBF3915005
:10AEA000504094F059F0882332F0660F771F881FC6
:10AEB00091505040C1F79E3F510544F7880F911DB6
:10AEC0009695879597F908955F3FACF0983E9CF072
:10AED000BB27869577956795B79508F4B1609395EC
:10AEE000C1F7BB0F58F711F460FFE8CF6F5F7F4FDA
:10AEF0008F4F9F4FE3CFB4CE0EF0DEC06CCE689480
:10AF000064CE93DEC8F39923D1F3C6F3DF93CF93D6
:10AF10001F930F93FF92C92FDD2788232AF02197D3
:10AF2000660F771F881FDAF720E030E040E85FEB1C
:10AF30009FE3883920F0803E30F021968F774BDDFB
:10AF4000E4E2F3E003C047DDE1E5F3E073DF8B010A
:10AF5000BE01EC01FB2E6F5771097595771F880BA9
:10AF6000990BD4DD28E132E741E35FE38FDEAF2DBB
:10AF70009801AE01FF900F911F91CF91DF913CDDC1
:10AF80003BCEFA01DC01AA0FBB1F9B01AC01BF57EE
:10AF900028F422273327442750781FC0B75188F45C
:10AFA000AB2F0024469537952795011CA395D2F326
:10AFB000002069F0220F331F441FB395DAF30DD040
:10AFC00009CD61307105A0E88A07B94630F49B01CC
:10AFD000AC016627772788279078309621F0208368
:10AFE00031834283538308950CD006CEFEDD40F0BA
:10AFF000F5DD30F021F45F3F19F0E7CD511130CE8F
:10B00000EACD0BDE98F39923C9F35523B1F3951BD1
:10B01000550BBB27AA2762177307840738F09F5F79
:10B020005F4F220F331F441FAA1FA9F333D00E2EE8
:10B030003AF0E0E830D091505040E695001CCAF755
:10B0400029D0FE2F27D0660F771F881FBB1F26171A
:10B0500037074807AB07B0E809F0BB0B802DBF01ED
:10B06000FF2793585F4F2AF09E3F510568F0ADCD02
:10B07000F7CD5F3FECF3983EDCF3869577956795C7
:10B08000B795F7959F5FC9F7880F911D969587959E
:10B0900097F90895E1E0660F771F881FBB1F6217BD
:10B0A00073078407BA0720F0621B730B840BBA0B7B
:10B0B000EE1F88F7E09508959F3F31F0915020F4FE
:10B0C000879577956795B795880F911D9695879584
:10B0D00097F90895DB018F939F930E94DF58BF91EA
:10B0E000AF91A29F800D911DA39F900DB29F900DD7
:10B0F00011240895A1E21A2EAA1BBB1BFD010DC04D
:10B10000AA1FBB1FEE1FFF1FA217B307E407F50717
:10B1100020F0A21BB30BE40BF50B661F771F881FF3
:10B12000991F1A9469F760957095809590959B0189
:10B13000AC01BD01CF010895052E97FB1EF40094CC
:10B140000E94B35857FD07D00E947A5807FC03D0DD
:10B150004EF40C94B35850954095309521953F4F3F
:10B160004F4F5F4F089590958095709561957F4FF3
:10B170008F4F9F4F0895EE0FFF1F0590F491E02D24
:10B1800019940E94C958332312F48A1B9B0B0C9408
:10B19000DA58A29FB001B39FC001A39F700D811D1B
:10B1A0001124911DB29F700D811D1124911D0895D0
:10B1B0000E94C958B7FF0895821B930B08950E94FF
:10B1C000C958A59F900DB49F900DA49F800D911D0F
:10B1D00011240895B7FF0C94DF580E94DF58821B9A
:10B1E000930B0895E894DF93CF93FC01DB010E9459
:10B1F000C9587F936F93E9019A01AC01BF93AF9354
:10B200003F932F93DF010E94C95826F46C1B7D0BDE
:10B21000820B930B9E01EB01FC010E942B59AF9115
:10B22000BF912F913F910E942B59BE01CF01F9018F
:10B230002F913F91CF91DF9108950790F691E02DE6
:10B240001BBE19942A0D3B1D4C1D5D1D6E1D7F1DDF
:10B25000801F911F08950E94C958460F571FC81F8D
:10B26000D91F08F431960895EF920F931F93CF934F
:10B27000DF93E80147FF02C034E101C034E0E42F6E
:10B28000FF27E7FDF095F7FF03C0F195E195F10980
:10B29000E32E022F2E2FAE010E946E5DCE01DF91B4
:10B2A000CF911F910F91EF900895CF93DF9382304C
:10B2B000910510F482E090E0E0913326F09134267D
:10B2C00020E030E0A0E0B0E0309739F140815181DA
:10B2D00048175907B8F04817590771F482819381CC
:10B2E000109729F012968D939C9313972CC08093FE
:10B2F00033269093342627C02115310531F04217AB
:10B30000530718F0A901DB0101C0EF019A01BD014B
:10B31000DF010280F381E02DD7CF21153105F9F04F
:10B32000281B390B2430310580F48A819B816115FB
:10B33000710521F0FB018283938304C0809333263F
:10B3400090933426FE01329644C0FE01E20FF31FB3
:10B350008193919322503109288339833AC02091F7
:10B36000312630913226232B41F420917E203091DA
:10B370007F20209331263093322620917C203091FB
:10B380007D202115310541F42DB73EB74091802035
:10B3900050918120241B350BE0913126F09132260B
:10B3A000E217F307A0F42E1B3F0B2817390778F09C
:10B3B000AC014E5F5F4F2417350748F04E0F5F1FFB
:10B3C00040933126509332268193919302C0E0E05E
:10B3D000F0E0CF01DF91CF910895CF93DF930097F5
:10B3E00009F487C0FC01329712821382C091332680
:10B3F000D0913426209781F420813181280F391F84
:10B4000080913126909132268217930779F5E09347
:10B410003126F09332266DC0DE0120E030E0AE1719
:10B42000BF0750F412964D915C9113979D01411501
:10B43000510509F1DA01F3CFA283B3834081518131
:10B44000840F951F8A179B0771F48D919C9111971A
:10B45000840F951F02968083918312968D919C9103
:10B460001397828393832115310529F4E0933326C2
:10B47000F09334263EC0D9011296ED93FC931397B6
:10B480004D915D91A40FB51FEA17FB0779F48081F8
:10B490009181840F951F0296D9018D939C931197EA
:10B4A0008281938112968D939C931397E0E0F0E054
:10B4B0008A819B81009719F0FE01EC01F9CFCE0142
:10B4C000029628813981820F931F20913126309175
:10B4D00032262817390769F4309729F41092332659
:10B4E0001092342602C012821382C0933126D09368
:10B4F0003226DF91CF9108958F929F92AF92BF92A3
:10B50000CF92DF92EF92FF92CF93DF93EC016881AD
:10B5100079818A819B81611571058105910521F4ED
:10B5200064E279ED8BE597E02DE133EF41E050E007
:10B530000E949C5849015A019B01AC01A7EAB1E461
:10B540000E94DF586B017C01ACEEB4EFA5019401C1
:10B550000E94ED58C60ED71EE81EF91EF7FE06C063
:10B5600081E0C81AD108E10880E8F80AC882D982C7
:10B57000EA82FB82C701B6019F77DF91CF91FF90EE
:10B58000EF90DF90CF90BF90AF909F908F900895F5
:10B590000C947C5A82E890E20C947C5A609382204E
:10B5A00070938320809384209093852008956F92D8
:10B5B0007F928F929F92AF92BF92CF92DF92EF9243
:10B5C000FF920F931F93CF93DF93EC01CB01209752
:10B5D00081F4DF91CF911F910F91FF90EF90DF9059
:10B5E000CF90BF90AF909F908F907F906F900C9472
:10B5F0005559FE01E60FF71F9E0122503109E2174F
:10B60000F30708F4ACC0D9010D911C9111970617EE
:10B610001707B8F00530110508F49FC0A801445081
:10B6200051094617570708F498C002501109061B24
:10B63000170B019311936D937C93CF010E94ED59E9
:10B640008CC05B01A01AB10A4E01800E911EA09120
:10B650003326B0913426612C712C60E070E0109795
:10B6600009F449C0A815B905C9F5ED90FC901197EA
:10B67000670142E0C40ED11CCA14DB0478F1470113
:10B680008A189B08640142E0C40ED11C1296BC903B
:10B6900012971396AC91B5E0CB16D10440F0B2826C
:10B6A000A38380829182D9018D939C9309C00E5F00
:10B6B0001F4F0E0D1F1DF90100831183EB2DFA2F73
:10B6C0006115710531F0DB011296ED93FC93139730
:10B6D00044C0E0933326F09334263FC06D917C91B3
:10B6E00011976616770608F43B01BD0112960D907E
:10B6F000BC91A02DB4CF609131267091322668158F
:10B700007905E9F468167906D0F440917C205091CF
:10B710007D204115510541F44DB75EB76091802001
:10B7200070918120461B570BE417F507C0F4E09396
:10B730003126F0933226F901808391830EC00E9456
:10B7400055597C01009759F0A801BE010E94135C75
:10B75000CE010E94ED59C70104C0CE0102C080E0B5
:10B7600090E0DF91CF911F910F91FF90EF90DF90CC
:10B77000CF90BF90AF909F908F907F906F900895E3
:10B78000662777270C94E65E1F93FC01992788278C
:10B79000BC01E89411911032E9F3193010F01E3019
:10B7A000C8F31B3251F01D3249F4689406C00E9460
:10B7B000BB5C610F711D811D911D119110531A30D9
:10B7C000B0F33EF490958095709561957F4F8F4FC3
:10B7D0009F4F1F910895911142C5803219F08950F1
:10B7E0008550D0F708959111089581548A5108F435
:10B7F000805E855A08959111089581568A5108F402
:10B80000805285580895FB01DC0105900D920020BF
:10B81000E1F70895FC0105900020E9F780959095E7
:10B820008E0F9F1F0895FB01DC0102C001900D9255
:10B8300041505040D8F708956817790768F4FB0124
:10B84000DC01E40FF51FA40FB51F02C002900E9299
:10B8500041505040D8F708950C94135CFC0181913D
:10B86000861721F08823D9F7992708953197CF01BA
:10B870000895FB01DC018D91019080190110D9F32D
:10B88000990B0895FB01DC0101900D920020E1F776
:10B890000895FB01DC014150504030F08D91019042
:10B8A000801919F40020B9F7881B990B0895FB0142
:10B8B000DC014150504048F001900D920020C9F742
:10B8C00001C01D9241505040E0F70895FC0181E015
:10B8D00090E00190061609F4CF010020D1F70197FE
:10B8E0000895FB0151915523A9F0BF01DC014D9151
:10B8F00045174111E1F759F4CD010190002049F0BD
:10B900004D9140154111C9F3FB014111EFCF81E089
:10B9100090E0019708954532510520F4423010F02F
:10B920000C94965CFB011082CB010895BB274A3032
:10B9300031F4992322F4BDE2909581959F4F0C94A8
:10B94000095D2532310520F4223010F00C94AC5CF6
:10B95000FA011082CA010895BB272A3051F49923B5
:10B9600042F4BDE290958095709561957F4F8F4F21
:10B970009F4F0C94DC5C592F482F372F262F660FD2
:10B98000771F881F991F660F771F881F991F620FE7
:10B99000731F841F951F660F771F881F991F0895B7
:10B9A0002532310520F4223010F00C94DB5CFA01D2
:10B9B0001082CA010895BB27FA01A62F62177105EC
:10B9C00081059105330B30FB66F0AA27660F771FC0
:10B9D000881F991FAA1FA21710F0A21B6395385049
:10B9E000A9F7A05DAA3308F0A95DA19336F7B111BC
:10B9F000B1931082CA010C944A614532510520F47A
:10BA0000423010F00C94085DFB011082CB010895C8
:10BA1000BB27FB015527AA27880F991FAA1FA41728
:10BA200010F0A41B83955051B9F7A05DAA3308F01C
:10BA3000A95DA193009779F7B111B1931192CB0150
:10BA40000C944A6103D0808199270895E0ECF1E0DD
:10BA5000378537FDFDCF348538603487FC01E050F1
:10BA6000F04F08950E94265D6081718182819381EB
:10BA700008950E94265D808191810895262FE0EC33
:10BA8000F1E0378537FDFDCF3485377F3487378543
:10BA900031FF09C036E3328738ED34BF31E03387F8
:10BAA000378537FDFDCF33E3328780839183128260
:10BAB000248325E3228728ED31E024BF33870196D4
:10BAC0000895242F0E943F5D252F0E943F5D0C9416
:10BAD000695D0E943E5D272F0C943F5D6F927F92BF
:10BAE0009F92AF92BF92CF92DF92EF92FF920F930D
:10BAF0001F93CF93DF93CDB7DEB72997CDBFDEBFBE
:10BB00006A01B22E102F0C3320F4FF24F394F00EB0
:10BB100002C04CE3F42E0F2D27E0AE014F5F5F4FC4
:10BB20000E9457607981272F2970213031F0E1FC84
:10BB300006C0E0FC06C060E005C06DE203C06BE239
:10BB400001C060E2AE2DA07173FF36C0662311F014
:10BB500084E001C083E08B1510F4B81A01C0B12C49
:10BB6000A1110BC0F6018B2D90E2882319F091935F
:10BB70008150FBCFCB0CD11CB12C662331F0F601E8
:10BB8000608396012F5F3F4F6901C6010396E2FE75
:10BB900005C02EE4F601208331E404C02EE6F60150
:10BBA000208331E631832283FC012B2D30E22223D6
:10BBB000F1F131932150FBCF72FF40C0662311F0A9
:10BBC00084E001C083E08B1510F4B81A01C0B12CD9
:10BBD000A1110BC0F6018B2D90E2882319F09193EF
:10BBE0008150FBCFCB0CD11CB12C662331F0F60178
:10BBF000608396012F5F3F4F6901C6010396E2FE05
:10BC000007C029E4F60120832EE4218326E406C040
:10BC100029E6F60120832EE6218326E62283FC0115
:10BC20002B2D30E2222319F031932150FBCFFC0160
:10BC3000EB0DF11D10828EEF9FEFB7C0B1E06111E7
:10BC400001C0B0E04B2F50E01816190624F49C01F7
:10BC50002F5F3F4F02C021E030E0240F351F11233A
:10BC600029F0412F50E04F5F5F4F02C040E050E0AD
:10BC7000420F531F2B2D30E04217530714F4B41A10
:10BC800001C0B12C2E2D287159F4F6012B2D30E274
:10BC9000222319F031932150FBCFCB0CD11CB12CB6
:10BCA000BB2331F0F601608396012F5F3F4F69019E
:10BCB000A1110BC0F6012B2D30E3222319F0319393
:10BCC0002150FBCFCB0CD11CB12CF80E0A81372FA1
:10BCD0003071A32E74FF03C0013309F4FA941F14CA
:10BCE0002CF42F2D293018F028E001C021E0682F16
:10BCF000392F97FF02C060E030E0462F532F612CB0
:10BD0000712C3EE2932EBC01621B71099B01DC0188
:10BD1000A41BB50BE1E0F0E0EC0FFD1FAE0FBF1F61
:10BD2000E12EF12CF194E194F1084F3FFFEF5F0712
:10BD300031F4F6019082B6016F5F7F4F6B0184177B
:10BD400095074CF02417350734F4BD01660D771DB7
:10BD5000FB01118101C010E341505109FFEF6F1A3F
:10BD60007F0AB6016F5F7F4F4E155F0524F0F60125
:10BD700010836B01DACF4817590739F4063320F4E2
:10BD8000053319F4A11001C011E3F6011083FB0182
:10BD90008B2D90E2882319F091938150FBCFFB010A
:10BDA000EB0DF11D108280E090E02996CDBFDEBF43
:10BDB000DF91CF911F910F91FF90EF90DF90CF9087
:10BDC000BF90AF909F907F906F9008958F929F92B9
:10BDD000AF92BF92CF92DF92EF92FF920F931F9399
:10BDE000CF93DF938B016115710521F0DB018C93FB
:10BDF00011969C93EC015E01BFEFAB1ABB0A750173
:10BE0000C8808C2D90E00E94EB5B892B11F0E5013E
:10BE1000F2CFEDE2CE1208C07E01F2E0EF0EF11C8F
:10BE2000C980DD24D39409C02BE2C21205C07E0173
:10BE300042E0E40EF11CC980D12CE701219743E0D8
:10BE400050E061E478E4CE010E943261892BC1F4B4
:10BE5000239645E050E06CE378E4CE010E94326125
:10BE6000892B09F425960115110519F0D801CD93F8
:10BE7000DC93D11006C160E070E080E89FE70AC162
:10BE800043E050E069E378E4CE010E943261892BFF
:10BE900059F40115110509F4F9C0B2E0EB0EF11CDB
:10BEA000F801E082F182F2C0F70160E070E0CB01BE
:10BEB000C0E0D0E07F01A0EDAA2EAC0C29E02A154D
:10BEC00030F14D2D4260B42E2D2D2870D2FE04C0CD
:10BED000211125C0219623C021112197A5E0B0E0B2
:10BEE0009B01AC010E94DF58660F771F881F991FC6
:10BEF0006A0D711D811D911D6839A9E97A078A07AC
:10BF0000A9E19A0760F0BD2DB660BB2E08C02EEFE8
:10BF1000A2120AC0D3FC50C04D2D4860B42E3196F9
:10BF2000D701CC90DB2CC6CF2C2D2F7D253409F0EA
:10BF300043C0A081AD3241F4BD2DB061DB2E7F0145
:10BF400022E0E20EF11C0CC07F01AB3231F04FEF6A
:10BF5000E41AF40A21E030E006C0A2E0EA0EF11C87
:10BF6000A18122E030E0A053AA3018F0E21AF30ACF
:10BF700023C0F70120E030E02038BCE03B075CF450
:10BF8000A901440F551F440F551F240F351F220FC1
:10BF9000331F2A0F311DAF014F5F5F4F7A01A08120
:10BFA000A053AA3010F4FA01E7CFD4FE03C03195B4
:10BFB00021953109C20FD31FD1FE09C0011511050A
:10BFC00031F0E1E0EE1AF108D801ED92FC920E9406
:10BFD00084552D2D2370233019F04B015C0106C0D0
:10BFE0004B015C01B7FAB094B7F8B09420E030E0B0
:10BFF000A901C501B4010E944F55882309F43EC030
:10C00000D7FF06C0D195C195D10908E518E402C053
:10C0100000E718E46801B8E1CB1AD10890E2E92EF4
:10C02000F12CCE15DF0574F0F8012591359145917D
:10C030005491C501B4010E943A564B015C01CE19DE
:10C04000DF09EFCF04501109F594E7940C151D0595
:10C0500041F78A2D880F8B2D881F8F3F49F020E0F4
:10C0600030E0A901C501B4010E944F55811106C0FD
:10C0700082E290E08093352690933626C501B40184
:10C0800009C060E070E080E89FEF04C060E070E00D
:10C0900080EC9FE7DF91CF911F910F91FF90EF9080
:10C0A000DF90CF90BF90AF909F908F9008952830F1
:10C0B00008F027E03327DA01990F311D87FD9160E1
:10C0C00000966105710539F432602E5F3D9330E3CF
:10C0D0002A95E1F708959F3F30F08038710561059A
:10C0E00009F03C5F3C5F3D93913008F08068911D02
:10C0F000DF93CF931F930F93FF92EF92192F987FA7
:10C100009695E92F96959695E90FFF27E253F74B01
:10C1100099273327EE24FF24A701E701059008940F
:10C12000079428F4360FE71EF81E491F511D660FAD
:10C13000771F881F991F0694A1F70590079428F48C
:10C14000E70EF81E491F561FC11D770F881F991F44
:10C15000661F0694A1F70590079428F4F80E491F6E
:10C16000561FC71FD11D880F991F661F771F069482
:10C17000A1F70590079420F4490F561FC71FD81F39
:10C18000990F661F771F881F0694A9F78491109551
:10C19000177041F0D695C79557954795F794E79452
:10C1A0001A95C1F7E4E7F8E4689415901591359174
:10C1B0006591959105907FE27395E118F10A430B23
:10C1C000560BC90BD009C0F7E10CF11E431F561FD7
:10C1D000C91FD01D7EF4703311F48A95E6CFE89420
:10C1E000015030F0080F0AF40027021708F4202F3E
:10C1F0002395022F7A3328F079E37D932A95E9F786
:10C2000010C07D932A9589F6069497956795379582
:10C2100017951794E118F10A430B560BC90BD00977
:10C2200098F023957E9173957A3308F070E37C93B0
:10C230002013B8F77E9170617D9330F0839571E3A0
:10C240007D9370E32A95E1F71124EF90FF900F9111
:10C250001F91CF91DF91992787FD90950895992798
:10C2600088270895FB01DC014150504088F08D91F2
:10C2700081341CF08B350CF4805E659161341CF0C8
:10C280006B350CF4605E861B611171F3990B089598
:10C29000881BFCCFDC01FC01672F71917723E1F74C
:10C2A000329704C07C916D9370836291AE17BF0783
:08C2B000C8F30895F894FFCFD4
:10C2B800010200010101010102020202020303035B
:10C2C800030404040405050506060607070808090B
:10C2D800090A0A0B0B0C0D0E0F1011121314151668
:10C2E8001718191A1B1C1D1F212325282B2E313521
:10C2F800383C401819141501010101010101010C14
:10C308000D0F0EFF07FF000000BF9906A914F90FD3
:10C31800D93E89439906490BF90FA9145919091EE1
:10C32800B9226927192CC9307935293A00003726EE
:10C338002000010000000301020300736176696EAA
:10C3480067207061746368200073697A65203D20F6
:10C3580000656E642061646472657373203D20001B
:10C368006C6F6164696E6720706174636820000097
:10C37800000000F73BFB3DA13BC93BB13BE93B6FEC
:06C388007666002E0000A5
:00000001FF
